:020000040000FA
:0400000007EF15F001
:0800080046EF15F0186E7F0BA6
:1000100018BC8008F76A240FF66E0800F55018BE69
:1000200000081200000306090C101316191C1F22E9
:1000300025282B2E313336393C3F414447494C4E1D
:10004000515355585A5C5E60626466686A6B6D6FA6
:1000500070717374757678797A7A7B7C7D7D7E7E1B
:100060007E7F7F7F7F002C6A2D6A01D0206E215019
:10007000205ED8A021062D502C5ED8A02D06D89049
:1000800021322032D8902D322C32031C1C6E041CDD
:100090001D6E1C2AD8B41D2A830E276E286A296A71
:1000A0002A6A2B6A266A0F0EEA6E02C0E9FF091C53
:1000B000D5EC02F000D000D0040020502826D8B0A3
:1000C000292A215029262C502A26D8B02B2A2D50F7
:1000D0002B2629509BDF800F196E2B5097DF800F46
:1000E00019261930262602C0E9FFEF500910D8A0C2
:1000F0000918EF6E2704D8B4830E276ED8B41C2AD3
:10010000D8B41D3ED7D71200086A800E346E89EF2E
:1001100000F0206A216A226A236A0A9AF2EC01F04E
:10012000D30FD8B40A8A2D0FC60FF8E20A0FF6E3F0
:100130001C6E1B6A1A6A196A0A0E186EB3EC02F07A
:100140001C501824206E1950216E000ED8B0010EDC
:1001500021261A50226E000ED8B0010E22261B5006
:10016000236E000ED8B0010E2326080606E0F2EC3E
:1001700001F0C60F02E20A0FDBE20AAA0BD0201E32
:10018000211E221E231E202AD8B4212AD8B4222AB6
:10019000D8B4232A20501200086A206E216A0096E3
:1001A0000850D8B40086050E076E270E1D6E100E7F
:1001B0000CD8030E1D6EE80E08D81D6A640E05D813
:1001C0001D6A0A0E02D8205008D01C6E2150196EEC
:1001D0002050186E9CEC02F01850186E074E0096D6
:1001E000085003E0075CD8B008D01850D8A4009697
:1001F00000B603D0300FE5EF01F01200366E2DAEE1
:1002000003D02D0EE5EC01F0106A116A126A136A30
:100210002D8E6A0E2C26D8902D322E322F3213328C
:100220001232113210322C3EF6D72F502C5C2F2672
:100230002C5E2E502D5C2E262D5E086A3AD82E0E8E
:10024000E5EC01F0376AD89010342F6E11342E6E21
:1002500012342D6E13342C6E3736D8902F362E363E
:100260002D362C36373610502F261150D8B0113C71
:100270002E261250D8B0123C2D261350D8B0133C65
:100280002C26D8B0373ED8902F362E362D362C3629
:1002900037363750300FE5EC01F02FC010F02EC08C
:1002A00011F02DC012F02CC013F0362ECBD7D89001
:1002B00012000096085003E100860A0E086E2FC057
:1002C0001BF02EC01AF02DC019F02CC018F0076AD0
:1002D000236A226A216A0A0E206E3FEC02F0072A86
:1002E0000750085CD8A4F4D72050D8A4009600A6E4
:1002F00002D0082C04D02050300FE5EC01F0082E7D
:10030000DED71200206E0750D8B4120020C0E9FFDB
:1003100021C0EAFFEF50D8B41200E5EC01F0204A0A
:10032000212A0706F0D7246E0F0EEA6EE26E025005
:10033000E96E120FE16E800E0A16080E256ED89037
:10034000D8B00A3E12D82432252EFAD7000029BA96
:100350000A300BD800D000D000D0D88006D8065084
:100360001D6E055025EC02F0120029AE0BD0EF50A7
:10037000091029AC0918EF6EE7500910D8A0091828
:10038000E76E0AD0EF500910D8A0091829BC091847
:10039000EF6E091CE71600D029501F0B000F196ED5
:1003A0002850110FD8B0192A000032EF02F0A66AC7
:1003B000A68E0900F55002E002D8FBD71200040017
:1003C0009EA8FDD7AD6ED880120001BA93EF01F060
:1003D00001B4DFEF01F001A205D001B003D001B2FA
:1003E000EE6E120034BEEE501200AA6AA96EA66A22
:1003F000A680A850A94AAA2A1200AA6AA86EA66ACC
:10040000A684550EA76EAA0EA76EA6820400A6B2F9
:10041000FDD7A694A94AAA2A1200E836E8363C0B72
:100420000109C212C009C216C050F80B0209C06E01
:10043000320E31EC02F0C2820400C2B2FDD7C4CF4A
:100440002DF0C3502C6E12001D6A1C6EFF0E1C2670
:100450001D2200D0D8A01200030E196EE70E02D89C
:10046000F5D7196AFD0F186EFF0E00D001D01826BF
:10047000040000D0D8A01926D8A01200F8D71B502D
:100480002318800BF46E1BAE06D0D880000E1856D1
:1004900019561A561B5623AE06D0D880000E205689
:1004A0002156225623561C6A1D6A1E6A1F6A306A2C
:1004B000316A326A336A235022102110201023E05F
:1004C000200EF36ED890183619361A361B36303691
:1004D0003136323633362050305C2150315822507C
:1004E00032582350335809E32050305E2150315A9E
:1004F0002250325A2350335AD8801C361D361E36AD
:100500001F36F32EDFD7F4AE06D0D880000E1C566F
:100510001D561E561F561CC018F01DC019F01EC0D7
:100520001AF01FC01BF030C020F031C021F032C0E3
:1005300022F033C023F01200216A206A100EF36EFD
:100540001934203621361C50205C1D50215805E3FB
:100550001C50205E1D50215AD88018361936F32EB3
:10056000EFD718501200200E246E306A316A326ABA
:10057000336AD89018A00ED0205030262150D8B021
:10058000213C31262250D8B0223C32262350D8B00C
:10059000233C332633323232313230321B321A327C
:1005A00019321832242EE5D71200E988E92AEC1610
:1005B0001200A66AA68E0900F55002E0EE6EFBD787
:1005C0001200F34E02D0E652FCD7E6CFEEFFE82E43
:1005D000FCD71200E466FED7F36EE552F32EFDD78A
:1005E000E6CFEEFFE82EFCD71200610EE75C05E6D1
:1005F0007B0EE75C02E7DF0EE716E650EE6EF5E1F4
:100600001200A66AA68EEE500900F55C02E1F566BE
:10061000FAD71200155011183A6E3ABE30D015BEF6
:1006200017D01450105CD8A0000CD8A4010C1550A1
:10063000115CD8A0000CD8A4010C1650125CD8A0F4
:10064000000CD8A4010C1750135CD8A0000C010CAE
:100650001050145CD8A0000CD8A4010C1150155CEB
:10066000D8A0000CD8A4010C1250165CD8A0000C25
:10067000D8A4010C1350175CD8A0000C010C11AECB
:10068000010C000C155011183A6E3ABE34D015BE4C
:1006900019D01450105CD8A0000CD8A4010C15502F
:1006A000115CD8A0000CD8A4010C1650125CD8A084
:1006B000000CD8A4010C1750135CD8A0000CD8A4CF
:1006C000010C000C1050145CD8A0000CD8A4010C34
:1006D0001150155CD8A0000CD8A4010C1250165C67
:1006E000D8A0000CD8A4010C1350175CD8A0000CA3
:1006F000D8A4010C000C11AE010C000C1450105CBD
:10070000376E19E2376C10C039F014C010F039C0E0
:1007100014F011C039F015C011F039C015F012C035
:1007200039F016C012F039C016F013C039F017C0F6
:1007300013F039C017F01A0E376078D0145276E0F3
:10074000366A1150396E15183B6E118E158E080ED3
:10075000375E08E317C036F016C017F015C016F064
:10076000156AF5D7372607E0D890153216321732BA
:100770003632372EF9D73BAE35D01750135E1650B0
:10078000125A1550115A07E2D880000E135612560D
:100790001156800E391A366C04E01306000E125AF8
:1007A000115A040E376E11660DD012C011F013C02D
:1007B00012F036C013F0366A080E105E2DE3372EA5
:1007C000F2D72AD011BE08D0D8903636133612365A
:1007D0001136102EF7D720D038AC26D036AE24D024
:1007E000366A11D0175013261650122215501122B6
:1007F00006E31132123213323632104A0FD038ACBF
:1008000013D036AE11D0133E0FD0123E0DD0113E94
:100810000BD0D8801390EDD7106A02D038821068C0
:10082000136A126A800E116E39AE119E13501200B7
:100830001150326E15183B6E145053E0105254E0B4
:10084000105E7F0E03E2102603E24DD010264EE22A
:1008500013C030F012C031F0328E158E180E396E82
:10086000136A126A116A0BD01750305C1650315857
:1008700011E3316E326A1750305E0BD004E215502E
:10088000325CF2E007E31750305E1650315A1550D3
:10089000325AD88013361236113630363136323667
:1008A000392EECD711BE07D010521DE03B32100696
:1008B000392A3B36E3D738AC1FD007E21750305EF9
:1008C0001650315A1550325A17E3133E15D0123EC6
:1008D00013D0113E11D0113212321332103E0CD00F
:1008E00005D0388604D03884106A02D03882106867
:1008F000136A126A800E116E3BAE119E13501200E5
:100900001150326E15183B6E1050D8A414503CE0B4
:1009100010267E0E03E3105E03E338D0105E33E34F
:1009200013C030F012C031F0328E158E136A126A85
:10093000116A180E396E32323132303206E31750F6
:100940001326165012221550112211321232133270
:10095000392EF1D711BE07D0133612361136105288
:1009600012E01006323438AC17D016E3133E14D020
:10097000123E12D0113E10D0D880113212321332F2
:10098000103E0AD003D03884106A02D03882106832
:10099000136A126A800E116E3BAE119E1350120044
:1009A000126A136A10C036F013C010F036C013F08C
:1009B00012C036F011C012F036C011F0960E396E2A
:1009C0003B6A10AE07D0D880000E1356125611564F
:1009D00010563B8E105218E038AC0DD013AE0BD031
:1009E000123E09D0113E07D0103E05D0D8801032FB
:1009F00011321232392A080E392612C013F011C0F2
:100A000012F010C011F015D0116613D0080E395E27
:100A1000125005E1080E395E135011E0136A116E91
:100A200013C012F0136A05D0D8901336123611365F
:100A3000390611AEF9D739C010F03BAE119E1350F4
:100A400012003D3D3D3D3D3D3D3D3D3D3D3D3D3D3E
:100A50003D3D3D3D3D3D3D3D3D3D3D3D3D3D3D3DC6
:100A60003D3D3D3D3D3D3D3D3D004E657720435084
:100A70005520636869702064657465637465642ECD
:100A800000003D3D3D3D3D3D3D3D3D3D3D3D3D3D10
:100A90003D3D3D3D3D3D3D3D3D3D3D3D3D3D3D3D86
:100AA0003D3D3D3D3D3D3D3D3D003D3D3D3D3D3DB3
:100AB0003D3D3D3D3D3D3D3D3D3D3D3D3D3D3D3D66
:100AC0003D3D3D3D3D3D3D3D3D3D3D3D3D3D3D3D56
:100AD0003D0053696572726120526164696F2053F1
:100AE000797374656D732054522053657175656E0A
:100AF000636572004669726D776172652076657212
:100B000073696F6E20002C206275696C6420000090
:100B10004E6574776F726B206164647265737320C5
:100B20002000456E746572202F2F68656C702066FA
:100B30006F7220636F6D6D616E642073756D6D6192
:100B4000727900003D3D3D3D3D3D3D3D3D3D3D3DDE
:100B50003D3D3D3D3D3D3D3D3D3D3D3D3D3D3D3DC5
:100B60003D3D3D3D3D3D3D3D3D3D3D00456E74655A
:100B70007220636F6D6D616E642000002F2F6F75A2
:100B8000743033206F6E00004641494C00004865C8
:100B90007921206E657720636F6D6D616E64000052
:100BA0006E65745F7061636B65742073686F756CDC
:100BB0006420626520636C656172203C00006E6594
:100BC000745F7061636B65745F6C656E203D2000BF
:100BD0007061636B6574203D20006E65745F73798E
:100BE0006E633D006E65745F747970653D006E657F
:100BF000745F66726F6D3D006E65745F746F3D006B
:100C00006E65745F6372633D00006E65745F706152
:100C1000796C6F61643D3C006E65745F7061636BFD
:100C200065745F6C656E3D006E65745F7061796CB4
:100C30006F61645F6C656E3D00002E2E2E20636830
:100C400065636B2074686520435243202E2E2E006E
:100C50006C656E677468206F6620617267203D2046
:100C6000000043616C63756C61746564204352439A
:100C7000203D20002C205061636B6574204352435B
:100C8000203D2000435243204661696C65642E205C
:100C900020426164207061636B657400435243209D
:100CA00050617373656420212020476F6F6420506A
:100CB00061636B6574006D79206164647265737340
:100CC0003D00484559212074686973207061636B49
:100CD000657420697320666F72206D6521004E6F08
:100CE00074206D79206164647265737300005365CC
:100CF0006E643A20000053656E643A20000053652C
:100D00006E643A20000053656E643A20000049206A
:100D10006861766520746865206E6574776F726BA4
:100D200020286E65745F61737365727420616374EB
:100D30006976652900004E6574776F726B20726565
:100D40006C656173656400004E6F77206174207478
:100D5000686520657865637574655F6E65745F634B
:100D60006F6D6D616E642073746570006E65745F85
:100D70007061636B65745F6C656E3D3D00002020A3
:100D8000636D645F64656C696D3D3D002020636D3B
:100D9000645F64656C696D3D3D3D0000636D645F3B
:100DA00064656C696D20203D0000636D645F636F56
:100DB0006D6D616E643D0000636D645F61726720FC
:100DC0002020203D00004F4E44454C415931000049
:100DD0004F4E44454C41593200004F4E44454C4122
:100DE000593300004F4E44454C41593400004F4E9A
:100DF00044454C41593500004F464644454C415905
:100E000031004F464644454C415932004F46464416
:100E1000454C415933004F464644454C41593400F6
:100E20004F464644454C41593500454E41424C459C
:100E3000000044495341424C45004E4F524D414CF5
:100E40004F4E00004F6E2073657175656E636520AF
:100E50003D206E6F726D616C0000524556455253D5
:100E6000454F4E004F6E2073657175656E6365204A
:100E70003D2072657665727365004E4F524D414C50
:100E80004F4646004F66662073657175656E6365F3
:100E9000203D206E6F726D616C0052455645525375
:100EA000454F464600004F66662073657175656E56
:100EB0006365203D207265766572736500004F554D
:100EC000543031004F55543032004F5554303300B8
:100ED0004F55543034004F5554303500494E310091
:100EE000494E3200494E3300435700004B455945A7
:100EF000520057504D00574D0000574D4C494D4939
:100F000054004144314D494E00004144324D494E58
:100F100000004144334D494E00004144344D494E98
:100F200000004144314D415800004144324D415888
:100F300000004144334D415800004144344D415874
:100F400000004144414C41524D00414443414C3129
:100F50000000414443414C320000414443414C3382
:100F60000000414443414C3400005345545245561F
:100F700000005345544255494C4400004E4554002E
:100F80004C4F43414C0048454C5000004C4F4144AD
:100F9000000053415645000053544154555300003E
:100FA00053544154450044454255474F4E00446513
:100FB000627567206D6F6465204F4E004445425551
:100FC000474F464600004465627567206D6F646553
:100FD000204F46460000535244454255474F4E006D
:100FE00053686966742072656769737465722064FA
:100FF00065627567206D6F6465204F4E0000535227
:1010000044454255474F4646000053686966742080
:101010007265676973746572206465627567206DB7
:101020006F6465204F4646004E455444454255473F
:101030004F4E00004E6574776F726B206465627569
:1010400067206D6F6465204F4E004E455444454205
:1010500055474F4646004E6574776F726B20646546
:10106000627567206D6F6465204F464600005049E9
:101070004E470000524F4C4C43414C4C0000464FF1
:101080005243454641494C0045594543414E445918
:101090000000455945004D534744495245435400CB
:1010A000536574206D657373616765206D6F64654A
:1010B00020746F206469726563742E004D53474E2F
:1010C00045540000536574206D6573736167652036
:1010D0006D6F646520746F206E6574776F726B201E
:1010E0007061636B6574206D6F64652E000045430D
:1010F000484F0000535441544554524947474552C4
:1011000000005245534554005245424F4F54000091
:1011100047455441444452005345544144445200CD
:101120005241440053494C454E5400004D4F4445F4
:101130000000424F4F5400002050494E473A2000D3
:101140002C2046726F6D3A2000002C20416464729E
:101150006573733A20005354415445313A00535457
:10116000415445313A005354415445313A005354A7
:10117000415445323A005354415445333A00535494
:10118000415445343A005354415445353A00535480
:10119000415445313A005354415445323A00535476
:1011A000415445333A005354415445343A00535462
:1011B000415445353A004F4B000053595354454D67
:1011C000204641494C2C2066726F6D3A20002E203B
:1011D000205368757474696E6720646F776E2E0093
:1011E0005365742050432075706461746520747277
:1011F000696767657220746F20004F4E00004B6571
:10120000796572206D6F6465204F4E004B6579657E
:1012100072206D6F6465204F464600005365742050
:10122000435720737065656420746F200000536518
:101230006E642043573A20002D2D2D2D2D20412F57
:101240004420434F4E5645525445522056414C552A
:101250004553202D2D2D2D2D2D2D2D2D0000416E92
:10126000616C6F6720696E2031203D200000762080
:101270002046776420202800416E616C6F672069EA
:101280006E2032203D20000076202052656620200E
:101290002800416E616C6F6720696E2033203D200D
:1012A000000076202020202020202800416E616C44
:1012B0006F6720696E2034203D20000076202020BA
:1012C0002020202028002D2D2D2D2D2D2D2D2D2DB4
:1012D0002D2D2D2D2D2D2D2D2D2D2D2D2D2D2D2D3E
:1012E0002D2D2D2D2D2D2D2D2D2D00004F4E00009F
:1012F000416E616C6F6720696E70757420616C61FE
:10130000726D206D6F6465204F4E00004F464600A1
:10131000416E616C6F6720696E70757420616C61DD
:10132000726D206D6F6465204F46460053657420D2
:10133000412F442031206D696E696D756D20746F89
:10134000200053657420412F442032206D696E695E
:101350006D756D20746F200053657420412F4420FB
:1013600033206D696E696D756D20746F2000536553
:101370007420412F442034206D696E696D756D2095
:10138000746F200053657420412F442031206D611B
:1013900078696D756D20746F200053657420412F3E
:1013A000442032206D6178696D756D20746F200066
:1013B00053657420412F442033206D6178696D7529
:1013C0006D20746F200053657420412F4420342019
:1013D0006D6178696D756D20746F200053657420A0
:1013E000412F4420696E70757420312063616C69EF
:1013F00062726174696F6E2076616C756520746FBE
:10140000200053657420412F4420696E707574204C
:10141000322063616C6962726174696F6E207661FB
:101420006C756520746F200053657420412F442033
:10143000696E70757420332063616C6962726174C7
:10144000696F6E2076616C756520746F200053653E
:101450007420412F4420696E7075742034206361BC
:101460006C6962726174696F6E2076616C7565205B
:10147000746F2000212121204C6F7720766F6C74CF
:1014800061676520616C61726D206F6E20696E709E
:1014900075742023302E20204D696E203D200000E1
:1014A000762E202041637475616C203D200021213F
:1014B00021204C6F7720766F6C7461676520616CBA
:1014C00061726D206F6E20696E7075742023312EED
:1014D00020204D696E203D200000762E20204163A3
:1014E0007475616C203D2000212121204C6F7720F4
:1014F000766F6C7461676520616C61726D206F6ED0
:1015000020696E7075742023322E20204D696E2064
:101510003D200000762E202041637475616C203DD3
:101520002000212121204C6F7720766F6C74616739
:101530006520616C61726D206F6E20696E707574CC
:101540002023332E20204D696E203D200000762E72
:10155000202041637475616C203D200021212120F1
:101560004F76657220766F6C7461676520616C617F
:10157000726D206F6E20696E7075742023302E207E
:10158000204D6178203D2000762E20204163747527
:10159000616C203D2000212121204F76657220764C
:1015A0006F6C7461676520616C61726D206F6E2075
:1015B000696E7075742023312E20204D6178203D96
:1015C0002000762E202041637475616C203D200040
:1015D000212121204F76657220766F6C74616765DA
:1015E00020616C61726D206F6E20696E7075742061
:1015F00023322E20204D6178203D2000762E2020A1
:1016000041637475616C203D2000212121204F76BB
:10161000657220766F6C7461676520616C61726DB4
:10162000206F6E20696E7075742023332E20204D3C
:101630006178203D2000762E202041637475616C16
:10164000203D20004F46460057617474206D65743C
:1016500065722070726F74656374696F6E2064695F
:101660007361626C656400004F4E000042617369F3
:10167000632077617474206D657465722070726F79
:1016800074656374696F6E20656E61626C65640079
:10169000435553544F4D0000456E61626C65207593
:1016A00073657220646566696E6564207761747421
:1016B000206D657465722070726F74656374696FF4
:1016C0006E2072616E6765004B657920696E70757A
:1016D0007420676F657320696E6163746976650055
:1016E0004B657920696E70757420676F6573206132
:1016F00063746976650053494C454E540000564565
:1017000052424F534500426F6F7420696E207665D8
:1017100072626F7365206D6F646500004F4E00004C
:1017200053696C656E74206D6F6465204F4646008A
:101730004C4F43414C004E4554574F524B00436170
:101740006C6C207369676E2073657420746F200061
:10175000536574206669726D776172652072657673
:1017600020746F200000536574206669726D776184
:101770007265206275696C6420746F2000004E658C
:1017800074776F726B206164647265737320736524
:101790007420746F2000536574206D79206E657419
:1017A000776F726B206164647265737320746F204D
:1017B0000000536574205478204F4E2064656C619E
:1017C00079203120746F2000536574205478204FA5
:1017D0004E2064656C6179203220746F200053655F
:1017E00074205478204F4E2064656C61792033203A
:1017F000746F2000536574205478204F4E20646528
:101800006C6179203420746F200053657420547803
:10181000204F4E2064656C6179203520746F200064
:101820005365742052782064656C6179203120748E
:101830006F2000005365742052782064656C6179D4
:10184000203220746F200000536574205278206489
:10185000656C6179203320746F200000536574201B
:1018600052782064656C6179203420746F20000008
:101870005365742052782064656C6179203520743A
:101880006F2000004F7574707574200020656E61C4
:10189000626C656400004F7574707574200020647C
:1018A000697361626C6564004F4E00004F464600EC
:1018B0005475726E206F75747075742031204F4EA0
:1018C00000005475726E206F75747075742031202D
:1018D0004F4646004F4E00004F4646005475726E0C
:1018E000206F75747075742032204F4E000054754F
:1018F000726E206F75747075742032204F464600EA
:101900004F4E00004F4646005475726E206F75743E
:101910007075742033204F4E00005475726E206F26
:1019200075747075742033204F4646004F4E00008A
:101930004F4646005475726E206F75747075742032
:1019400034204F4E00005475726E206F75747075A0
:10195000742034204F4646004F4E00004F4646004C
:101960005475726E206F75747075742035204F4EEB
:1019700000005475726E206F757470757420352078
:101980004F4646004F4E00004F4646005475726E5B
:1019900020696E7075742031204F4E005475726E40
:1019A00020696E7075742031204F464600004F4EFE
:1019B00000004F4646005475726E20696E70757453
:1019C0002032204F4E005475726E20696E7075740F
:1019D0002032204F464600004F4E00004F46460042
:1019E0005475726E20696E7075742033204F4E00EE
:1019F0005475726E20696E7075742033204F4646A0
:101A00000000526573657420616C6C2070617261B6
:101A10006D657465727320746F2064656661756CA2
:101A2000742076616C7565732E00436F6E6669670E
:101A300075726174696F6E20736176656420746F6E
:101A400020666C617368206D656D6F72792E000081
:101A5000436F6E66696775726174696F6E206C6F33
:101A6000616465642066726F6D20666C61736820C6
:101A70006D656D6F72792E002D2D2D2054522053DF
:101A80007175656E63657220436F6D6D616E647311
:101A9000202D2D2D2D2D2D2D2D2D2D2D2D2D2D2D83
:101AA0002D2D2D2D2D2D2D2D2D2D2D2D2D2D2D2D66
:101AB0002D2D2D004F4E44454C4159306E2078203D
:101AC000206D732E2044656C617920782028312D9B
:101AD0003530303029206D732E206265666F726557
:101AE000207475726E696E67206F6E206F757470EA
:101AF000757420236E2C20207768657265206E2017
:101B00003D20312D35004F464644454C4159306EFD
:101B10002078206D732E2044656C61792078202810
:101B2000312D3530303029206D732E206265666F7F
:101B30007265207475726E696E67206F6666206FBD
:101B4000757470757420236E2C207768657265201B
:101B50006E203D20312D35004E4F524D414C4F4EA1
:101B60002020202020202020205475726E206F6EAF
:101B70002020696E206E6F726D616C20207365711C
:101B800075656E63652C20312C20322C20332C207F
:101B9000342C203520202844656661756C7429003A
:101BA0004E4F524D414C4F464620202020202020B1
:101BB000205475726E206F666620696E206E6F729B
:101BC0006D616C202073657175656E63652C2035C1
:101BD0002C20342C20332C20322C2031202028445F
:101BE000656661756C742900524556455253454FE0
:101BF0004E20202020202020205475726E206F6EF1
:101C00002020696E20726576657273652073657138
:101C100075656E63652C20352C20342C20332C20E8
:101C2000322C20310000524556455253454F46460E
:101C3000202020202020205475726E206F666620A0
:101C4000696E20726576657273652073657175655E
:101C50006E63652C20312C20322C20332C20342C28
:101C600020350000454E41424C4520782020202060
:101C70002020202020456E61626C6573206F757492
:101C800070757420782028312D352900444953413E
:101C9000424C4520782020202020202020446973B9
:101CA00061626C6573206F7574707574207820287C
:101CB000312D352900002D2D2D2041646D696E20B8
:101CC000436F6D6D616E6473202D2D2D2D2D2D2D87
:101CD0002D2D2D2D2D2D2D2D2D2D2D2D2D2D2D2D34
:101CE0002D2D2D2D2D2D2D2D2D2D2D2D2D2D2D2D24
:101CF0002D2D000048454C50202020202020202061
:101D00002020202020446973706C617920746869F8
:101D1000732068656C7020696E666F726D6174699E
:101D20006F6E000053544154555320202020202032
:101D30002020202020446973706C617920746865CC
:101D40002063757272656E7420636F6E6669677565
:101D5000726174696F6E00004C4F41442020202056
:101D60002020202020202020204C6F616420636FE1
:101D70006E66696775726174696F6E2066726F6DE9
:101D800020666C617368206D656D6F7279005341D8
:101D900056452020202020202020202020202053B5
:101DA00061766520636F6E66696775726174696FCD
:101DB0006E20746F20666C617368206D656D6F7244
:101DC00079005245534554202020202020202020F7
:101DD0002020205265736574206F7065726174698C
:101DE0006E6720706172616D657465727320746FC7
:101DF000207374616E646172642064656661756CE1
:101E0000742076616C75657300005245424F4F54E3
:101E100020202020202020202020205265626F6F6B
:101E200074207468652073797374656D0000424F87
:101E30004F542053494C454E5420202020202054FC
:101E400075726E73206F666620626F6F74206D65A9
:101E5000737361676500424F4F5420564552424F9D
:101E6000534520202020205475726E73206F6E2001
:101E7000626F6F74206D6573736167650000535402
:101E80004154455452494747455220787878205567
:101E90007064617465732050432070726F67726163
:101EA0006D20646973706C61792069662064656C6B
:101EB0006179206973203E207878782028646566EF
:101EC00061756C74203D20323530206D732900001F
:101ED0002D2D2D20412F4420436F6E766572746541
:101EE00072202D20416E616C6F6720496E70757491
:101EF0002043616C6962726174696F6E2D2D2D2DA6
:101F00002D2D2D2D2D2D2D2D2D2D2D2D0000414430
:101F100043414C6E207878782020202020202041DA
:101F20006473206F722073756274726163747320BE
:101F3000746865206F6666736574207878782028E9
:101F4000696E206D696C69766F6C74732920746F8B
:101F50002074686520412F4420636F6E766572742B
:101F6000657220276E27202028312D342900414416
:101F70006E4D494E20787878202020202020205354
:101F8000657473206C6F772074726967676572205F
:101F9000616C61726D20766F6C7461676520746F1F
:101FA0002078787820766F6C74732028696E20769C
:101FB0006F6C7473290041446E4D415820787878D5
:101FC00020202020202020536574732068696768D2
:101FD000207472696767657220616C61726D20762A
:101FE0006F6C7461676520746F2078787820766FE5
:101FF0006C74732028696E20766F6C7473290000EE
:102000005241442020202020202020202020202059
:10201000205265616420616E616C6F6720696E702B
:10202000757420766F6C74616765206E6F77000041
:102030002D2D2D2057617474204D657465722043D9
:102040006F6D6D616E6473202D2D2D2D2D2D2D2D19
:102050002D2D2D2D2D2D2D2D2D2D2D2D2D2D2D2DB0
:102060002D2D2D2D2D2D2D2D2D2D2D2D0000574DB0
:10207000204F4E20202020202020202020202054CF
:1020800075726E206F6E2062617369632077617470
:1020900074206D65746572206D6F6E69746F7269FE
:1020A0006E672E202048696768207265666C6563DC
:1020B00074656420706F7765722064697361626C07
:1020C00065732073657175656E6365720000574DA9
:1020D000204F464620202020202020202020205451
:1020E00075726E206F666620626173696320776126
:1020F0007474206D65746572206D6F6E69746F7293
:10210000696E672E0000574D20435553544F4D20A4
:10211000202020202020205475726E206F6E2077A2
:10212000617474206D65746572206D6F6E69746F73
:1021300072696E672E2020496E6869626974207327
:10214000657175656E6365207768656E207265667A
:102150006C656374656420766F6C74616765206874
:102160006974732074686520574D4C494D4954205B
:1021700076616C756500574D4C494D49542078780F
:10218000782020202020204D696E696D756D2072A9
:1021900065666C656374656420766F6C74616765F1
:1021A00020746861742077696C6C20696E6869625C
:1021B0006974207468652073657175656E63650068
:1021C0002D2D2D20435720436F6D6D616E6473205C
:1021D0002D2D2D2D2D2D2D2D2D2D2D2D2D2D2D2D2F
:1021E0002D2D2D2D2D2D2D2D2D2D2D2D2D2D2D2D1F
:1021F0002D2D2D2D2D2D2D2D2D2D2D2D00004B4533
:10220000594552204F4E20202020202020202054AD
:1022100075726E206F6E206B65796572206D6F64CC
:10222000652E20204F757470757420352077696C89
:102230006C2073656E64204357207573696E672048
:1022400074686520435720636F6D6D616E64000094
:102250004B45594552204F46462020202020202023
:10226000205475726E206F6666206B6579657220EA
:102270006D6F64652E20204F757470757420352045
:1022800077696C6C206F70657261746520696E206F
:102290006E6F726D616C2073657175656E636572CA
:1022A000206D6F6465004357207878787878202017
:1022B0002020202020202053656E642074657874CF
:1022C00020787878787820696E2043572075736974
:1022D0006E67206F7574707574203520696E206B81
:1022E00065796572206D6F64650057504D20787870
:1022F00020202020202020202020205365742043EF
:102300005720737065656420696E20617070726F0C
:1023100078696D61746520776F726473207065727F
:10232000206D696E7574652028312D3939290000BA
:102330002D2D2D204E6574776F726B20436F6D6D60
:10234000616E6473202D2D2D2D2D2D2D2D2D2D2DD8
:102350002D2D2D2D2D2D2D2D2D2D2D2D2D2D2D2DAD
:102360002D2D2D2D2D2D2D2D2D2D2D2D00005345B9
:1023700054414444522078782020202020202057A7
:1023800068657265207878206973207468652062BA
:102390006F6172642773206E6574776F726B206152
:1023A00064647265737320286265747765656E2056
:1023B0003120616E64203135290047455441444441
:1023C00052202020202020202020204765742074C7
:1023D00068652076616C7565206F6620746865207D
:1023E000626F6172642773206E6574776F726B2001
:1023F000616464726573730053494C454E54204FB9
:102400004E2020202020202020446F206E6F74203A
:1024100073656E64206D6573736167657320746F97
:102420002073657269616C20706F727420776865C3
:102430006E207374617465206368616E67657300F4
:1024400053494C454E54204F464620202020202002
:102450002053656E64206D657373616765732074C6
:102460006F2073657269616C20706F727420776879
:10247000656E207374617465206368616E6765734F
:1024800000004D534744495245435420202020200A
:1024900020202053657420726573706F6E73652001
:1024A000746F20706C61696E207465787420666F3B
:1024B000726D617400004D53474E4554202020201A
:1024C0002020202020202053657420726573706FB7
:1024D0006E736520746F206E6574776F726B2070F9
:1024E00061636B657420666F726D617400002D2DE1
:1024F0002D204D616E75616C204F75747075742060
:10250000436F6D6D616E6473202D2D2D2D2D2D2D3E
:102510002D2D2D2D2D2D2D2D2D2D2D2D2D2D2D2DEB
:102520002D2D2D2D2D2D2D2D2D2D00004F555430C1
:102530006E204F4E2020202020202020204D616E34
:1025400075616C6C79207475726E204F4E20206F0F
:102550007574707574206E2028312D3529004F5503
:1025600054306E204F464620202020202020204D31
:10257000616E75616C6C79207475726E204F464681
:10258000206F7574707574206E2028312D352900E8
:102590002D2D2D20496E7465726E616C204465622C
:1025A000756767696E6720436F6D6D616E64732038
:1025B0002D2D2D2D2D2D2D2D2D2D2D2D2D2D2D2D4B
:1025C0002D2D2D2D2D2D2D2D2D2D2D2D0000444566
:1025D0004255474F4E2020202020202020202054EC
:1025E00075726E206F6E20646562756767696E67CD
:1025F000206D657373616765730044454255474FAD
:1026000046462020202020202020205475726E2055
:102610006F666620646562756767696E67206D65C1
:102620007373616765730000464F524345464149E5
:102630004C2020202020202020466F7263657320CC
:10264000756E697420696E746F204641494C206D27
:102650006F64652E20205368757473206F66662042
:10266000616C6C206F757470757473003D3D3D3DF9
:102670003D5B2043555252454E5420434F4E4649F0
:102680004755524154494F4E205D3D3D3D3D3D3DF6
:102690003D3D3D00436F6E66696720636F64652052
:1026A000203A2000426F61726420747970652020A6
:1026B000203A200046572076657273696F6E20209D
:1026C000203A20004657206275696C642020202043
:1026D000203A20004D792061646472657373202074
:1026E000203A20004F4E202064656C617920312013
:1026F000203A20004F4E202064656C617920322002
:10270000203A20004F4E202064656C6179203320F0
:10271000203A20004F4E202064656C6179203420DF
:10272000203A20004F4E202064656C6179203520CE
:10273000203A20004F46462064656C6179203120A4
:10274000203A20004F46462064656C617920322093
:10275000203A20004F46462064656C617920332082
:10276000203A20004F46462064656C617920342071
:10277000203A20004F46462064656C617920352060
:10278000203A20003A20456E61626C6564003A2070
:1027900044495341424C454400004F757470757470
:1027A00020312020202020003A20456E61626C6597
:1027B00064003A2044495341424C454400004F755F
:1027C0007470757420322020202020003A20456E3D
:1027D00061626C6564003A2044495341424C45446F
:1027E00000004F7574707574203320202020200065
:1027F0003A20456E61626C6564003A204449534159
:10280000424C454400004F7574707574203420208C
:10281000202020003A20456E61626C6564003A20F9
:1028200044495341424C454400004F7574707574DF
:1028300020352020202020004F4E207365717565C3
:102840006E636520203A204E6F726D616C004F4EB2
:102850002073657175656E636520203A2052657638
:102860006572736564004F46462073657175656EC9
:102870006365203A204E6F726D616C004F464620B2
:1028800073657175656E6365203A20526576657271
:1028900073656400435720737065656420202020B1
:1028A000203A200057617474206D6574657220634E
:1028B0006865636B696E67204F46460053696D70AB
:1028C0006C652077617474206D657465722063682F
:1028D00065636B696E6720656E61626C656400009C
:1028E00057617474206D65746572206C696D6974CC
:1028F0002073657420746F200000414420616C6176
:10290000726D206D6F64653A204F66660000414429
:1029100020616C61726D206D6F64653A204F4E00CE
:10292000416E616C6F672031206D696E203A200026
:102930002020202020202020206D6178203A2000B7
:1029400020202020202020202063616C203A2000BD
:10295000416E616C6F672032206D696E203A2000F5
:102960002020202020202020206D6178203A200087
:1029700020202020202020202063616C203A20008D
:10298000416E616C6F672033206D696E203A2000C4
:102990002020202020202020206D6178203A200057
:1029A00020202020202020202063616C203A20005D
:1029B000416E616C6F672034206D696E203A200093
:1029C0002020202020202020206D6178203A200027
:1029D00020202020202020202063616C203A20002D
:1029E000436F6D6D206D6F6465202020203A204C70
:1029F0006F63616C0000436F6D6D206D6F646520C7
:102A00002020203A204E6574776F726B0000F86AC0
:102A1000400E386E006A030EAF6E200EAC6E900E44
:102A2000AB6E2EEE81F094988298949A829A93904D
:102A300081909392819293948194110E05012E6F4F
:102A4000C70E2D6F510E2C6F810E2B6F0101D99D7A
:102A5000D98F040E196EB00E186E1D6A90C51CF049
:102A60009CEC02F005018E6F19C08FF5030E8D6F7F
:102A7000520E8C6F05EEDCF0540EEE6E520EEE6EC2
:102A8000310EEE6EEF6A00017DEF15F09EAA23D0A5
:102A9000060EAB141DE1E2CF3DF0E1CF3CF03E2A43
:102AA000FF0E3E5C01E33E6A1DEE82F03E50E126E1
:102AB000000EE222AECFE7FF0D0EE75C02E1010E51
:102AC000426E3EC017F43DC0E2FF3CC0E1FF110082
:102AD000AB98AB8800D011003E6A3F6A9D8AC00E59
:102AE000F26E12009D9A0DEE82F0FF0EEE6AE82E55
:102AF000FDD73E6A3F6A9D8A1200400EAF6E900E6F
:102B0000AB6E200EAC6E0B0EC16EF19E320E24EC3D
:102B100002F08298829A8190819281949394819418
:102B20009392819293908190949A829A94988298A9
:102B30000101D99BD9BF8282D9AF829205012A9126
:102B40000101CC6BD46BDB6BDA6B01EEDCF04F0E6A
:102B5000EE6E4B0EEE6EEF6A01EE1CF0EE6A01EEC9
:102B6000E1F0EE6A0401A06B640E9F6FA26BA16B93
:102B700004EE19F0300EEE6EEE6EEF6A0601098972
:102B8000098B099D0401A36B04EEA4F0EE6A050114
:102B9000276B266BE689E68BE68DE68F06010981B9
:102BA00009930501776BCD0E7B6FCC0E7A6F4C0EBF
:102BB000796F7C0E786F0601099509970101686BA2
:102BC0006A6B0501256B4A6B496B486B476B4E6B13
:102BD0004D6B4C6B4B6B526B516B506B4F6B566B21
:102BE000556B546B536B01016B6B05015A6B596B41
:102BF000586B576B5E6B5D6B5C6B5B6B626B616B99
:102C0000606B5F6B666B656B646B636B6A6B696B48
:102C1000700E686F830E676F6E6B6D6B700E6C6FEE
:102C2000830E6B6F726B716B700E706F830E6F6FB4
:102C3000766B756B700E746F830E736F01016C6B26
:102C40004BDF00012AEC18F00101D991D993D995F5
:102C5000010E0501E36F010ED76FD96B040ED86F1B
:102C6000DB6B210EDA6F010EE56F5A6B596B586BF7
:102C7000576B6A6B696B200E686F810E676F5E6BB6
:102C80005D6B5C6B5B6B6E6B6D6B200E6C6F810EA6
:102C90006B6F626B616B606B5F6B726B716B200E45
:102CA000706F810E6F6F666B656B646B636B766BB9
:102CB000756B200E746F810E736FE697296B640E2F
:102CC000286FE329E46F0001C3EC29F082B66AEFB4
:102CD00016F0F9D794908280000EF5EC01F0050112
:102CE000D76FD7290001D8A4A1EF16F00401A35390
:102CF0000001D8A4A1EF16F004EEA4F00A0EF76EBE
:102D0000420EF66ED9EC02F0EF6A25EC1EF004EEEE
:102D1000A4F00A0EF76E6A0EF66ED9EC02F0EF6AB6
:102D200025EC1EF0D3EC42F072EC43F004EEA4F07C
:102D30000A0EF76E820EF66ED9EC02F0EF6A25EC01
:102D40001EF091EC46F0F8EC37F001EE6DF0020E5B
:102D5000016E0501E551CCEC00F0EF6A010E0401B3
:102D6000A353D8A4000E356E010E01016B53D8A4F5
:102D7000000E35140001D8B433EF17F004EEA4F0C0
:102D80000A0EF76EAA0EF66ED9EC02F0EF6A25EC89
:102D90001EF004EEA4F00A0EF76ED20EF66ED9EC19
:102DA00002F0EF6A25EC1EF004EEA4F00A0EF76EB6
:102DB000F40EF66ED9EC02F0020E016E086AD9C567
:102DC00021F0D8C520F0CFEC00F00B0EF76E060E08
:102DD000F66ED9EC02F0020E016E086ADBC521F036
:102DE000DAC520F0CFEC00F0EF6A25EC1EF004EE1F
:102DF000A4F00B0EF76E100EF66ED9EC02F0020E78
:102E0000016E0501E551CCEC00F0EF6A04EEA4F090
:102E10000B0EF76E220EF66ED9EC02F0EF6A00018F
:102E200025EC1EF004EEA4F00B0EF76E440EF66EC9
:102E3000D9EC02F0EF6A25EC1EF004EEA4F00B0EC4
:102E4000F76E6C0EF66ED9EC02F0EF6A25EC1EF010
:102E500004EEA4F00B0EF76E7C0EF66ED9EC02F0C9
:102E6000EF6A0BEC1EF0320E24EC02F0949082908C
:102E70000B0EF76E880EF66E01EEDCF001EC03F03F
:102E8000D8A445EF17F024EC2AF0D896060109AD36
:102E9000D8860001D8B64FEF17F084EF17F001EE97
:102EA000A0F0020E016EE86A80BA010ECCEC00F0D0
:102EB000EF6A01EEA0F084EC00F0808AE8A0809A2E
:102EC00001EEB5F0020E016EE86A81B6010ECCEC9F
:102ED00000F0EF6A01EEB5F084EC00F08186E8A026
:102EE00081961AEC2FF0010E01016C5D0001D8A44F
:102EF0007CEF17F0DCEC34F0050177530001D8B417
:102F000084EF17F083EC37F00601099D000181A8DA
:102F10008CEF17F0EAEF17F0010E0101CC6FE86AB1
:102F200080BA010E356EE86A81B6010E35100001D7
:102F3000D8B4A0EF17F00101CC6B0001A3EF17F09C
:102F4000010E0101CC6F0001010E0101CC5D010EEB
:102F5000D8A4000E356E010E05012ABDE86A3514AD
:102F60000001D8B4B6EF17F08BEF3DF0010E010170
:102F7000CC5D010ED8A4000E356EE86A05012ABDAD
:102F8000010E35140001D8B4C8EF17F009EF38F07E
:102F9000010E0101CC53D8A4000E356E010E0501BF
:102FA0002ABDE86A35140001D8B4D9EF17F0CCEF88
:102FB0003AF0010E0101CC53D8A4000E356EE86A38
:102FC00005012ABD010E35140001D8B4EAEF17F04F
:102FD00090EF3DF00501264B272B2651285D275108
:102FE00029590001D8B013EF18F00501276B266BA3
:102FF000D8962AB1D8860001D8B606EF18F0050198
:103000002A8194928292000113EF18F0D89605015C
:103010002AA1D8860001D8B612EF18F005012A912E
:103020009492828200010401A1519F5DA251A05996
:103030000001D8B021EF18F02AEC18F00401A26BBF
:10304000A16B0001010E425CD8A429EF18F02EEC10
:1030500018F00ED7426A72EC15F01200D8960101F2
:10306000D9A5D8860001D8B642EF18F00B0EF76E3E
:103070008E0EF66ED7EC01F00D0EDFEC01F00A0EAD
:10308000DFEC01F001EEE1F0820EEE6AE82EFDD7F2
:10309000D8960101D9A5D8860001D8B666EF18F0F8
:1030A0000B0EF76EA00EF66ED7EC01F001EEE1F01C
:1030B000EE5003E0DFEC01F0FBD73E0EDFEC01F059
:1030C0000D0EDFEC01F00A0EDFEC01F03E0404010E
:1030D000176F00013EAE6FEF18F00401176B00018F
:1030E000D8960101D9A5D8860001D8B68AEF18F084
:1030F0000B0EF76EBE0EF66ED7EC01F0040E016EED
:1031000004011751CCEC00F00D0EDFEC01F00A0EBB
:10311000DFEC01F00001040117530001D8A494EF83
:1031200018F0010E0401176F0001040117050B6E62
:103130000101CC6B00010101CC510B5C0001D8A056
:10314000DAEF18F0D8960101CCAFD8860001D8B6D6
:10315000ACEF18F00101CC6B00010101CC290DEEA0
:1031600082F0E926000EEA22EFCF0FF001EEE1F047
:10317000CC51E926000EEA220FC0EFFFD896D9A560
:10318000D8860001D8B6D4EF18F0040E016E01EE17
:10319000E1F00101CC51E926000EEA22EF50CCEC1F
:1031A00000F0200EDFEC01F000010101CC2B00014A
:1031B000D8A4C0D7DDEC18F0120001EEE1F011EE5A
:1031C000E1F0F5EC02F0D8960101D9A5D88600010E
:1031D000D8B6FEEF18F00B0EF76ED00EF66ED7ECE9
:1031E00001F001EEE1F0EE5003E0DFEC01F0FBD77F
:1031F0000D0EDFEC01F00A0EDFEC01F002EE63F0E1
:1032000011EEE1F0010EF36E010EE1EC02F0EF6A57
:10321000D8960101D9A5D8860001D8B623EF19F0B8
:103220000B0EF76EDA0EF66ED7EC01F002EE63F0DD
:10323000EE5003E0DFEC01F0FBD70D0EDFEC01F008
:103240000A0EDFEC01F002EE65F011EEE1F0020E85
:10325000F36E010EE1EC02F0EF6AD8960101D9A5F8
:10326000D8860001D8B648EF19F00B0EF76EE40EC1
:10327000F66ED7EC01F002EE65F0EE5003E0DFEC05
:1032800001F0FBD70D0EDFEC01F00A0EDFEC01F0D0
:1032900002EE68F011EEE1F0030EF36E020EE1ECC7
:1032A00002F0EF6AD8960101D9A5D8860001D8B6F8
:1032B0006DEF19F00B0EF76EEE0EF66ED7EC01F017
:1032C00002EE68F0EE5003E0DFEC01F0FBD70D0EEC
:1032D000DFEC01F00A0EDFEC01F002EE6CF011EE13
:1032E000E1F0050EF36E020EE1EC02F0EF6AD89603
:1032F0000101D9A5D8860001D8B692EF19F00B0EBE
:10330000F76EF80EF66ED7EC01F002EE6CF0EE50B0
:1033100003E0DFEC01F0FBD70D0EDFEC01F00A0E4D
:10332000DFEC01F002EE70F011EEE1F0070EF36E4B
:10333000030EE1EC02F0EF6AD8960101D9A5D88618
:103340000001D8B6B7EF19F00C0EF76E000EF66E4E
:10335000D7EC01F002EE70F0EE5003E0DFEC01F08C
:10336000FBD70D0EDFEC01F00A0EDFEC01F002EEF0
:1033700075F011EEE1F00A0EF36E090E0401175D0F
:10338000E1EC02F0EF6AD8960101D9A5D8860001D8
:10339000D8B6E1EF19F00C0EF76E0A0EF66ED7EC08
:1033A00001F002EE75F0EE5003E0DFEC01F0FBD728
:1033B0003E0EDFEC01F00D0EDFEC01F00A0EDFEC4B
:1033C00001F001EEE1F0E86AEE5202E0E83EFCD7DF
:1033D0000401176FD8960101D9A5D8860001D8B687
:1033E00004EF1AF00C0EF76E180EF66ED7EC01F023
:1033F000040E016E04011751CCEC00F00D0EDFEC51
:1034000001F00A0EDFEC01F0000102EE75F0E86A4F
:10341000EE5202E0E83EFCD70401186FD896010195
:10342000D9A5D8860001D8B628EF1AF00C0EF76E91
:10343000280EF66ED7EC01F0040E016E040118514F
:10344000CCEC00F00D0EDFEC01F00A0EDFEC01F029
:10345000000104EE19F012EE68F0030EE75204E0EA
:10346000E6CFEEFFE82EFAD7EF6A300E0201655D77
:103470000001D8A43EEF1AF0E2EF1BF02F0E02017C
:10348000655D0001D8A447EF1AF00101D98B000156
:103490002F0E0201655D0001D8A454EF1AF004EE6E
:1034A00019F0300EEE6EEF6A2F0E0201655D00011D
:1034B000D8A45DEF1AF0AFEC1FF02F0E0201655D8E
:1034C0000001D8A469EF1AF001016A6B00016CEFEA
:1034D0001AF0010E01016A6F00012F0E0201655DF5
:1034E0000001D8A475EF1AF01200D8960101D9A5F1
:1034F000D8860001D8B689EF1AF00C0EF76E3A0E96
:10350000F66ED7EC01F00D0EDFEC01F00A0EDFECE9
:1035100001F0D8960101D9A5D8860001D8B6A3EF4D
:103520001AF00C0EF76E500EF66ED7EC01F0040E8A
:10353000016E0101D451CCEC00F00D0EDFEC01F076
:103540000A0EDFEC01F000010401166B010E01010F
:10355000CC6F0001060E0101CC5D0001D8B00DEF6B
:103560001BF001EEE1F00101CC51E926000EEA2248
:10357000EF50D46FD4510401161B01EEA0F0020EDF
:10358000016E0101CC51CCEC00F0EF6A01EEB5F018
:10359000020E016E04011651CCEC00F0EF6AD896D1
:1035A0000101D9A5D8860001D8B607EF1BF001EEBE
:1035B000A0F0EE5003E0DFEC01F0FBD7200EDFECD3
:1035C00001F001EEE1F00101CC51E926000EEA2202
:1035D000EF50DFEC01F0200EDFEC01F0630EDFECCA
:1035E00001F0720EDFEC01F0630EDFEC01F03D0E36
:1035F000DFEC01F001EEB5F0EE5003E0DFEC01F09E
:10360000FBD70D0EDFEC01F00A0EDFEC01F000013C
:103610000101CC2B0001D8A49CD7090E0101CC6F6D
:1036200000010101CC510401175D0001D8A075EF24
:103630001BF001EEE1F00101CC51E926000EEA2277
:10364000EF500B6E0B500401161B01EEA0F0020EA2
:10365000016E0101CC51CCEC00F0EF6A01EEB5F047
:10366000020E016E04011651CCEC00F0EF6AD89600
:103670000101D9A5D8860001D8B66FEF1BF001EE85
:10368000A0F0EE5003E0DFEC01F0FBD7200EDFEC02
:1036900001F001EEE1F00101CC51E926000EEA2231
:1036A000EF50DFEC01F0200EDFEC01F0630EDFECF9
:1036B00001F0720EDFEC01F0630EDFEC01F03D0E65
:1036C000DFEC01F001EEB5F0EE5003E0DFEC01F0CD
:1036D000FBD70D0EDFEC01F00A0EDFEC01F000016C
:1036E0000101CC2B0001D8A49BD7D8960101D9A504
:1036F000D8860001D8B69CEF1BF00C0EF76E620E58
:10370000F66ED7EC01F0040E016E04011651CCECFC
:1037100000F00C0EF76E740EF66ED7EC01F002EEB0
:1037200070F0EE5003E0DFEC01F0FBD70D0EDFECA4
:1037300001F00A0EDFEC01F0000102EE70F084EC03
:1037400000F00B6E21C00CF022C00DF023C00EF073
:103750000D500E100AE10C500D1007E10B50040142
:1037600016190001D8B4CEEF1BF0D8960101D9A5E7
:10377000D8860001D8B6C9EF1BF00C0EF76E840E88
:10378000F66ED7EC01F00D0EDFEC01F00A0EDFEC67
:1037900001F02AEC18F01200E2EF1BF0D8960101BC
:1037A000D9A5D8860001D8B6E2EF1BF00C0EF76E53
:1037B0009C0EF66ED7EC01F00D0EDFEC01F00A0E58
:1037C000DFEC01F0D8960101D9A5D8860001D8B662
:1037D000FCEF1BF00C0EF76EB60EF66ED7EC01F098
:1037E000040E016E0501E551CCEC00F00D0EDFEC8E
:1037F00001F00A0EDFEC01F0000102EE6CF084EC47
:1038000000F00101D46FD76BD4510501E55D0001D3
:10381000D8A40EEF1CF0010E0101D76F0001630E5A
:103820000101D45D0001D8A419EF1CF0010E0101C3
:10383000D76F0001630E0101D45D0001D8A424EF0D
:103840001CF0020E01016A6F0001010E0101D75D3B
:103850000001D8A44AEF1CF0D8960101D9A5D8865A
:103860000001D8B640EF1CF00C0EF76EC20EF66EDB
:10387000D7EC01F00D0EDFEC01F00A0EDFEC01F0E9
:1038800002EE75F012EE75F0F5EC02F0C6EC1FF0EA
:103890005EEF1CF0D8960101D9A5D8860001D8B6F4
:1038A0005EEF1CF00C0EF76EDE0EF66ED7EC01F03C
:1038B0000D0EDFEC01F00A0EDFEC01F02AEC18F03F
:1038C000120002EECAF011EE31F0360EE75204E0BB
:1038D000E6CFEEFFE82EFAD7EF6A72EC1CF01AEC96
:1038E0001FF0120003EE0CF0820EEE6AE82EFDD7F8
:1038F00002EEB7F02F0EEE6EEF6A02EEBAF0410E56
:10390000EE6EEF6A02EEBDF0020E016E0501E551AA
:10391000CCEC00F0EF6A02EEBDF0E86AEE5202E095
:10392000E83EFCD70B6E010E0B5C0001D8A4A9EF9A
:103930001CF001EEB5F0300EEE6E12EEBDF0030E8F
:10394000E75204E0E6CFEEFFE82EFAD7EF6AB5EFD4
:103950001CF001EEB5F012EEBDF0030EE75204E0EC
:10396000E6CFEEFFE82EFAD7EF6A02EEBDF011EED9
:10397000B5F0140EE75204E0E6CFEEFFE82EFAD7DA
:10398000EF6A02EEC1F014EE19F0030EE75204E004
:10399000E6CFEEFFE82EFAD7EF6A02EEC1F0E86A52
:1039A000EE5202E0E83EFCD70101D46FD45300018F
:1039B000D8A4E1EF1CF002EEC1F0300EEE6EEE6E18
:1039C000EF6A010E0101D45D0001D8A402EF1DF0E1
:1039D00004EEA4F0300EEE6E12EEC1F0030EE752CC
:1039E00004E0E6CFEEFFE82EFAD7EF6A02EEC1F070
:1039F00014EEA4F0800EE75204E0E6CFEEFFE82ECE
:103A0000FAD7EF6A020E0101D45D0001D8A40FEFCE
:103A10001DF002EEC1F0EE50FEE1ED52EF6A01EE54
:103A20006DF012EEB7F0020EE75204E0E6CFEEFFC3
:103A3000E82EFAD712EEBAF0020EE75204E0E6CF13
:103A4000EEFFE82EFAD712EEBDF0030EE75204E0C7
:103A5000E6CFEEFFE82EFAD712EEC1F0030EE752E2
:103A600004E0E6CFEEFFE82EFAD712EECAF0410EE0
:103A7000E75204E0E6CFEEFFE82EFAD7EF6A01EE58
:103A80006DF0E86AEE5202E0E83EFCD70101D86F23
:103A9000D76B01EE6DF0E86AEE5202E0E83EFCD72B
:103AA0000B6E010ECC6F00010101CC510B5C0001CB
:103AB000D8A077EF1DF001EE6DF00101CC51EB5075
:103AC000D46FD451D71B01EEA0F0020E016ECC5181
:103AD000CCEC00F0EF6A01EEB5F0020E016ED751AA
:103AE000CCEC00F0EF6ACC2B0001D8A4DCD702EEBE
:103AF000C5F0020E016E0101D751CCEC00F0EF6A67
:103B000002EEC5F0E86AEE5202E0E83EFCD7D46F60
:103B1000010ED45D0001D8A49DEF1DF004EEA4F0C9
:103B2000300EEE6EEE6E12EEC5F0040EE75204E0BB
:103B3000E6CFEEFFE82EFAD7EF6A020E0101D45D60
:103B40000001D8A4B2EF1DF004EEA4F0300EEE6E2A
:103B500012EEC5F0040EE75204E0E6CFEEFFE82EC9
:103B6000FAD7EF6A030E0101D45D0001D8A4C5EFB6
:103B70001DF004EEA4F012EEC5F0040EE75204E0CE
:103B8000E6CFEEFFE82EFAD7EF6A02EEC5F014EEAC
:103B9000A4F0800EE75204E0E6CFEEFFE82EFAD75D
:103BA000EF6A03EE0CF012EEB7F0020EE75204E0FB
:103BB000E6CFEEFFE82EFAD712EEBAF0020EE75289
:103BC00004E0E6CFEEFFE82EFAD712EEBDF0030ECA
:103BD000E75204E0E6CFEEFFE82EFAD712EEC1F08E
:103BE000030EE75204E0E6CFEEFFE82EFAD712EE1E
:103BF000C5F0040EE75204E0E6CFEEFFE82EFAD758
:103C000012EECAF0410EE75204E0E6CFEEFFE82ED6
:103C1000FAD7EF6A1200800E026E100E096E400E87
:103C2000296E540E286E066A056A200E016E810EFA
:103C3000076E040E216EA40E82EC01F00D0E93ECC3
:103C400001F00A0E93EC01F0120001016A53000129
:103C5000D8A473EF1EF04FEC1FF0D8960101D9A540
:103C6000D8860001D8B648EF1EF00C0EF76EEE0EA7
:103C7000F66ED7EC01F004EEA4F0EE5003E0DFECBA
:103C800001F0FBD70D0EDFEC01F00A0EDFEC01F0C6
:103C90000401A3530001D8A45BEF1EF004EEA4F0CE
:103CA000EE5003E0DFEC01F0FBD70D0EDFEC01F08E
:103CB0000A0EDFEC01F0010E0401A35D0001D8A49F
:103CC0006FEF1EF004EEA4F0EE5003E0DFEC01F025
:103CD000FBD70D0EDFEC01F00A0EDFEC01F098ECE3
:103CE0001FF019EF1FF0010E01016A5D0001D8A459
:103CF000C2EF1EF04FEC1FF0D8960101D9A5D8866F
:103D00000001D8B697EF1EF00C0EF76EF60EF66EA9
:103D1000D7EC01F004EEA4F0EE5003E0DFEC01F08C
:103D2000FBD70D0EDFEC01F00A0EDFEC01F0040111
:103D3000A3530001D8A4AAEF1EF004EEA4F0EE50A5
:103D400003E0DFEC01F0FBD70D0EDFEC01F00A0E13
:103D5000DFEC01F0010E0401A35D0001D8A4BEEF69
:103D60001EF004EEA4F0EE5003E0DFEC01F0FBD710
:103D70000D0EDFEC01F00A0EDFEC01F098EC1FF005
:103D800019EF1FF0020E01016A5D0001D8A419EFBE
:103D90001FF00501E551320DF3CF1CF0F4CF1DF0FB
:103DA00026EC02F000014FEC1FF0D8960101D9A5D6
:103DB000D8860001D8B6F0EF1EF00C0EF76EFE0E9E
:103DC000F66ED7EC01F004EEA4F0EE5003E0DFEC69
:103DD00001F0FBD70D0EDFEC01F00A0EDFEC01F075
:103DE0000401A3530001D8A403EF1FF004EEA4F0D4
:103DF000EE5003E0DFEC01F0FBD70D0EDFEC01F03D
:103E00000A0EDFEC01F0010E0401A35D0001D8A44D
:103E100017EF1FF004EEA4F0EE5003E0DFEC01F02A
:103E2000FBD70D0EDFEC01F00A0EDFEC01F098EC91
:103E30001FF012004FEC1FF0D8960101D9A5D886CB
:103E40000001D8B637EF1FF00D0EF76E060EF66EB6
:103E5000D7EC01F003EE0CF0EE5003E0DFEC01F0E4
:103E6000FBD70D0EDFEC01F00A0EDFEC01F0D89667
:103E7000060109B7D8860001D8B64CEF1FF003EE53
:103E80000CF0EE5003E0DFEC01F0FBD70D0EDFECA1
:103E900001F00A0EDFEC01F098EC1FF012000101B6
:103EA000D76B000101EEA0F0020E016EE86A82B647
:103EB000010ECCEC00F0EF6A01EEA0F084EC00F013
:103EC0000101D46F010ED45D0001D8A46AEF1FF088
:103ED0007EEF1FF00101D72B0501E5510A0DF3CF4D
:103EE0001CF0F4CF1DF026EC02F0330E0101D75D7B
:103EF0000001D8A07DEF1FF01200D3D794908280EC
:103F0000050E24EC02F0D8960101D9A5D88600014F
:103F1000D8B697EF1FF00D0EF76E0E0EF66ED7ECBB
:103F200001F00D0EDFEC01F00A0EDFEC01F01200E3
:103F300094908290D8960101D9A5D8860001D8B670
:103F4000AEEF1FF00D0EF76E360EF66ED7EC01F0E9
:103F50000D0EDFEC01F00A0EDFEC01F01200D89636
:103F60000101D9ABD8860001D8B6C5EF1FF002EE2B
:103F700075F011EEE1F0030EF36E000E0401175D13
:103F8000E1EC02F0EF6A0101D99B0001D896010132
:103F9000D9A5D8860001D8B6DAEF1FF00D0EF76E5E
:103FA000480EF66ED7EC01F00D0EDFEC01F00A0EB4
:103FB000DFEC01F001EEE1F012EE75F0410EE75298
:103FC00004E0E6CFEEFFE82EFAD7EF6A416A01EE91
:103FD000E1F0E86AEE5202E0E83EFCD70401176F18
:103FE0000101CC6B00010101CC510401175D0001FE
:103FF000D8A07EEF20F0D8960101D9A5D88600017F
:10400000D8B615EF20F00D0EF76E6C0EF66ED7ECED
:1040100001F0040E016E04011751CCEC00F00D0EFE
:10402000DFEC01F00A0EDFEC01F00001D89601018F
:10403000D9A5D8860001D8B63BEF20F0690EDFEC99
:1040400001F03D0EDFEC01F0DFEC01F0040E016E3B
:104050000101CC51CCEC00F00D0EF76E7E0EF66E29
:10406000D7EC01F04150CCEC00F00D0EDFEC01F08C
:104070000A0EDFEC01F0000101EEE1F00101CC518C
:10408000E926000EEA22EF500B6E200E0B5C0001B9
:10409000D8A451EF20F00101CC29416E00017EEF40
:1040A00020F0D8960101D9A5D8860001D8B678EFBE
:1040B00020F0690EDFEC01F03D0EDFEC01F0DFECEB
:1040C00001F0DFEC01F0040E016E0101CC51CCECEB
:1040D00000F00D0EF76E8C0EF66ED7EC01F041502D
:1040E000CCEC00F00D0EDFEC01F00A0EDFEC01F07D
:1040F00000010101CC2B0001D8A474D700EE43F0DD
:1041000011EEE1F04104E6CFEEFFE82EFCD7EF6AB6
:1041100000EE43F010EE43F0F5EC02F000EE58F044
:1041200011EEE1F041500401175DEAEC02F0EF6A94
:1041300041520001D8A4A0EF20F000EE58F0EE6A42
:1041400000EE58F010EE58F0F5EC02F001EE31F010
:1041500010EE58F0400EE75204E0E6CFEEFFE82EF6
:10416000FAD7EF6AD8960101D9A5D8860001D8B64A
:10417000CBEF20F00D0EF76E9C0EF66ED7EC01F033
:10418000040E016E4150CCEC00F00D0EDFEC01F09E
:104190000A0EDFEC01F0D8960101D9A5D8860001FE
:1041A000D8B6E6EF20F00D0EF76EAA0EF66ED7EC3D
:1041B00001F000EE43F0EE5003E0DFEC01F0FBD73E
:1041C0000D0EDFEC01F00A0EDFEC01F0D8960101D4
:1041D000D9A5D8860001D8B601EF21F00D0EF76EF3
:1041E000B80EF66ED7EC01F000EE58F0EE5003E09A
:1041F000DFEC01F0FBD70D0EDFEC01F00A0EDFEC77
:1042000001F00D0EF76EC60EF66E00EE43F001ECF7
:1042100003F0D8A410EF21F0ADEC3EF0E6EF25F06E
:104220000D0EF76ED00EF66E00EE43F001EC03F0CB
:10423000D8A41FEF21F0D3EC3EF0E6EF25F00D0EF1
:10424000F76EDA0EF66E00EE43F001EC03F0D8A440
:104250002EEF21F0F9EC3EF0E6EF25F00D0EF76EB3
:10426000E40EF66E00EE43F001EC03F0D8A43DEF4F
:1042700021F01FEC3FF0E6EF25F00D0EF76EEE0E8D
:10428000F66E00EE43F001EC03F0D8A44CEF21F001
:1042900045EC3FF0E6EF25F00D0EF76EF80EF66EEA
:1042A00000EE43F001EC03F0D8A45BEF21F06BECDF
:1042B0003FF0E6EF25F00E0EF76E020EF66E00EE02
:1042C00043F001EC03F0D8A46AEF21F091EC3FF049
:1042D000E6EF25F00E0EF76E0C0EF66E00EE43F0D4
:1042E00001EC03F0D8A479EF21F0B7EC3FF0E6EF52
:1042F00025F00E0EF76E160EF66E00EE43F001EC92
:1043000003F0D8A488EF21F0DDEC3FF0E6EF25F0D4
:104310000E0EF76E200EF66E00EE43F001EC03F089
:10432000D8A497EF21F003EC40F0E6EF25F00E0E55
:10433000F76E2A0EF66E00EE43F001EC03F0D8A4FF
:10434000A6EF21F029EC40F0E6EF25F00E0EF76E17
:10435000320EF66E00EE43F001EC03F0D8A4B5EF98
:1043600021F08FEC40F0E6EF25F00E0EF76E3A0EDE
:10437000F66E00EE43F001EC03F0D8A4D0EF21F08C
:104380000601098904EEA4F00E0EF76E440EF66ED7
:10439000D9EC02F0EF6A000125EC1EF0E6EF25F003
:1043A0000E0EF76E5A0EF66E00EE43F001EC03F0BF
:1043B000D8A4EBEF21F00601099904EEA4F00E0E4B
:1043C000F76E640EF66ED9EC02F0EF6A000125EC90
:1043D0001EF0E6EF25F00E0EF76E7A0EF66E00EE8A
:1043E00043F001EC03F0D8A406EF22F00601098B9C
:1043F00004EEA4F00E0EF76E840EF66ED9EC02F009
:10440000EF6A000125EC1EF0E6EF25F00E0EF76EC8
:104410009A0EF66E00EE43F001EC03F0D8A421EF03
:1044200022F00601099B04EEA4F00E0EF76EA60E14
:10443000F66ED9EC02F0EF6A000125EC1EF0E6EF13
:1044400025F00E0EF76EBE0EF66E00EE43F001EC98
:1044500003F0D8A430EF22F0F5EC40F0E6EF25F0C1
:104460000E0EF76EC40EF66E00EE43F001EC03F094
:10447000D8A43FEF22F02AEC41F0E6EF25F00E0E33
:10448000F76ECA0EF66E00EE43F001EC03F0D8A40E
:104490004EEF22F05FEC41F0E6EF25F00E0EF76EE6
:1044A000D00EF66E00EE43F001EC03F0D8A45DEF01
:1044B00022F094EC41F0E6EF25F00E0EF76ED60EEA
:1044C000F66E00EE43F001EC03F0D8A46CEF22F09E
:1044D000C9EC41F0E6EF25F00E0EF76EDC0EF66E3D
:1044E00000EE43F001EC03F0D8A47BEF22F001ECE6
:1044F00042F0E6EF25F00E0EF76EE00EF66E00EEDF
:1045000043F001EC03F0D8A48AEF22F001EC42F072
:10451000E6EF25F00E0EF76EE40EF66E00EE43F0B9
:1045200001EC03F0D8A499EF22F047EC42F0E6EF5B
:1045300025F00E0EF76EE80EF66E00EE43F001EC7D
:1045400003F0D8A4A8EF22F014EC2BF0E6EF25F04E
:104550000E0EF76EEC0EF66E00EE43F001EC03F07B
:10456000D8A4B7EF22F023EC2BF0E6EF25F00E0EE7
:10457000F76EF20EF66E00EE43F001EC03F0D8A4F5
:10458000C6EF22F04DEC2BF0E6EF25F00E0EF76EA5
:10459000F60EF66E00EE43F001EC03F0D8A4D5EF72
:1045A00022F035EC37F0E6EF25F00E0EF76EFA0E3E
:1045B000F66E00EE43F001EC03F0D8A4E4EF22F035
:1045C000E1EC37F0E6EF25F00F0EF76E020EF66E17
:1045D00000EE43F001EC03F0D8A4F3EF22F0B0ECCE
:1045E00031F0E6EF25F00F0EF76E0A0EF66E00EED4
:1045F00043F001EC03F0D8A402EF23F0EBEC31F030
:10460000E6EF25F00F0EF76E120EF66E00EE43F099
:1046100001EC03F0D8A411EF23F026EC32F0E6EF22
:1046200025F00F0EF76E1A0EF66E00EE43F001EC59
:1046300003F0D8A420EF23F061EC32F0E6EF25F090
:104640000F0EF76E220EF66E00EE43F001EC03F053
:10465000D8A42FEF23F09CEC32F0E6EF25F00F0EFC
:10466000F76E2A0EF66E00EE43F001EC03F0D8A4CC
:104670003EEF23F0D7EC32F0E6EF25F00F0EF76EA9
:10468000320EF66E00EE43F001EC03F0D8A44DEFCD
:1046900023F012EC33F0E6EF25F00F0EF76E3A0E32
:1046A000F66E00EE43F001EC03F0D8A45CEF23F0CB
:1046B0004DEC33F0E6EF25F00F0EF76E420EF66E7E
:1046C00000EE43F001EC03F0D8A46BEF23F07BEC99
:1046D00031F0E6EF25F00F0EF76E4A0EF66E00EEA3
:1046E00043F001EC03F0D8A47AEF23F088EC33F028
:1046F000E6EF25F00F0EF76E520EF66E00EE43F069
:1047000001EC03F0D8A489EF23F0DDEC33F0E6EF01
:1047100025F00F0EF76E5A0EF66E00EE43F001EC28
:1047200003F0D8A498EF23F032EC34F0E6EF25F054
:104730000F0EF76E620EF66E00EE43F001EC03F022
:10474000D8A4A7EF23F087EC34F0E6EF25F00F0EA6
:10475000F76E6A0EF66E00EE43F001EC03F0D8A49B
:10476000B6EF23F03EEC3EF0E6EF25F00F0EF76ECD
:10477000720EF66E00EE43F001EC03F0D8A4C5EF24
:1047800023F05CEC3EF0E6EF25F00F0EF76E7C0EAA
:10479000F66E00EE43F001EC03F0D8A4D4EF23F062
:1047A0009AEC2AF0E6EF25F00F0EF76E800EF66E0B
:1047B00000EE43F001EC03F0D8A4E3EF23F092EC19
:1047C0002AF0E6EF25F00F0EF76E860EF66E00EE7D
:1047D00043F001EC03F0D8A4F2EF23F0B7EC4FF074
:1047E000E6EF25F00F0EF76E8C0EF66E00EE43F03E
:1047F00001EC03F0D8A401EF24F091EC46F0E6EFD1
:1048000025F00F0EF76E920EF66E00EE43F001ECFF
:1048100003F0D8A410EF24F072EC43F0E6EF25F09B
:104820000F0EF76E980EF66E00EE43F001EC03F0FB
:10483000D8A41FEF24F05BEC4AF0E6EF25F00F0E52
:10484000F76EA00EF66E00EE43F001EC03F0D8A474
:104850002EEF24F0A5EC26F0E6EF25F00F0EF76E14
:10486000A60EF66E00EE43F001EC03F0D8A449EF7B
:1048700024F00101D98104EEA4F00F0EF76EAE0E04
:10488000F66ED9EC02F0EF6A000125EC1EF0E6EFBF
:1048900025F00F0EF76EBC0EF66E00EE43F001EC45
:1048A00003F0D8A464EF24F00101D99104EEA4F040
:1048B0000F0EF76EC60EF66ED9EC02F0EF6A00012D
:1048C00025EC1EF0E6EF25F00F0EF76ED60EF66E15
:1048D00000EE43F001EC03F0D8A47FEF24F00101D7
:1048E000D98304EEA4F00F0EF76EE00EF66ED9EC4D
:1048F00002F0EF6A000125EC1EF0E6EF25F00F0E46
:10490000F76EFE0EF66E00EE43F001EC03F0D8A455
:104910009AEF24F00101D99304EEA4F0100EF76E83
:104920000A0EF66ED9EC02F0EF6A000125EC1EF0DB
:10493000E6EF25F0100EF76E280EF66E00EE43F04F
:1049400001EC03F0D8A4B5EF24F00101D98504EE01
:10495000A4F0100EF76E340EF66ED9EC02F0EF6A8A
:10496000000125EC1EF0E6EF25F0100EF76E4A0E62
:10497000F66E00EE43F001EC03F0D8A4D0EF24F083
:104980000101D99504EEA4F0100EF76E560EF66EE6
:10499000D9EC02F0EF6A000125EC1EF0E6EF25F0FD
:1049A000100EF76E6E0EF66E00EE43F001EC03F0A3
:1049B000D8A4DFEF24F0EDEC25F0E6EF25F0100EA3
:1049C000F76E740EF66E00EE43F001EC03F0D8A41F
:1049D000EEEF24F020EC26F0E6EF25F0100EF76E57
:1049E0007E0EF66E00EE43F001EC03F0D8A4FDEF6E
:1049F00024F018EC2AF0E6EF25F0100EF76E880E82
:104A0000F66E00EE43F001EC03F0D8A40CEF25F0B5
:104A1000C0EC2AF0E6EF25F0100EF76E920EF66E5F
:104A200000EE43F001EC03F0D8A41BEF25F0C0EC3E
:104A30002AF0E6EF25F0100EF76E960EF66E00EEF9
:104A400043F001EC03F0D8A436EF25F00401A36B8A
:104A500004EEA4F0100EF76EA00EF66ED9EC02F084
:104A6000EF6A000125EC1EF0E6EF25F0100EF76E60
:104A7000BC0EF66E00EE43F001EC03F0D8A452EF4A
:104A800025F0010E0401A36F04EEA4F0100EF76EE2
:104A9000C40EF66ED9EC02F0EF6A000125EC1EF0B0
:104AA000E6EF25F0100EF76EEE0EF66E00EE43F018
:104AB00001EC03F0D8A461EF25F061EC1CF0E6EF07
:104AC00025F0100EF76EF40EF66E00EE43F001ECDA
:104AD00003F0D8A470EF25F0A2EC2AF0E6EF25F061
:104AE000110EF76E020EF66E00EE43F001EC03F0CD
:104AF000D8A47FEF25F0D3EC42F0E6EF25F0110EBD
:104B0000F76E080EF66E00EE43F001EC03F0D8A449
:104B10008EEF25F086EF15F0E6EF25F0110EF76E1B
:104B2000100EF66E00EE43F001EC03F0D8A49DEFFA
:104B300025F07AEC3EF0E6EF25F0110EF76E180E38
:104B4000F66E00EE43F001EC03F0D8A4ACEF25F0D4
:104B50008FEC3EF0E6EF25F0110EF76E200EF66EAC
:104B600000EE43F001EC03F0D8A4BBEF25F0B9EC64
:104B700030F0E6EF25F0110EF76E240EF66E00EE23
:104B800043F001EC03F0D8A4CAEF25F0C7EC3DF0E8
:104B9000E6EF25F0110EF76E2C0EF66E00EE43F0E8
:104BA00001EC03F0D8A4D9EF25F0EBEC3DF0E6EFF3
:104BB00025F0110EF76E320EF66E00EE43F001ECAA
:104BC00003F0D8A4E6EF25F09EEC3DF00401A26BC3
:104BD000A16B00012AEC18F0120002EECAF0110ECF
:104BE000F76E380EF66ED9EC02F011EEDCF0040E22
:104BF000E75204E0E6CFEEFFE82EFAD7110EF76E8B
:104C0000400EF66ED9EC02F015EEDCF0060EE7521F
:104C100004E0E6CFEEFFE82EFAD7110EF76E4A0E4B
:104C2000F66ED9EC02F0020E016E0501E551CCECF6
:104C300000F0EF6A000172EC1CF01AEC1FF0120099
:104C40000501E5510A0DF3CF1CF0F4CF1DF026EC61
:104C500002F00001C2DF12000401A3530001D8A436
:104C600066EF26F002EECAF0110EF76E560EF66EE3
:104C7000D9EC02F0020E016EE86A82B8010ECCECAB
:104C800000F0020E016EE86A82BA010ECCEC00F070
:104C9000020E016EE86A81B0010ECCEC00F0020E4B
:104CA000016EE86A81B2010ECCEC00F0020E016EDA
:104CB000E86A81B4010ECCEC00F0300EEE6EEE6EC0
:104CC000EE6EEF6A72EC1CF01AEC1FF0010E04019C
:104CD000A35D0001D8A4A1EF26F002EECAF0110EE8
:104CE000F76E5E0EF66ED9EC02F0020E016EE86A07
:104CF00082B8010ECCEC00F0020E016EE86A82BAB6
:104D0000010ECCEC00F0020E016EE86A81B0010EDB
:104D1000CCEC00F0020E016EE86A81B2010ECCEC20
:104D200000F0020E016EE86A81B4010ECCEC00F0D6
:104D3000300EEE6EEE6EEE6EEF6A72EC1CF01AEC58
:104D40001FF0140E24EC02F012000401A353000122
:104D5000D8A433EF28F002EECAF0110EF76E660EFB
:104D6000F66ED9EC02F0020E016EE86A82B8010E0E
:104D7000CCEC00F0020E016EE86A82BA010ECCECB7
:104D800000F0020E016EE86A81B0010ECCEC00F07A
:104D9000020E016EE86A81B2010ECCEC00F0020E48
:104DA000016EE86A81B4010ECCEC00F0300EEE6EBC
:104DB000EE6EEE6EEF6A72EC1CF01AEC1FF0140E41
:104DC00024EC02F002EECAF0110EF76E6E0EF66ED3
:104DD000D9EC02F0020E016E3AC52FF039C52EF063
:104DE00038C52DF037C52CF0030EFEEC00F02C0E6C
:104DF000EE6E020E016E3EC52FF03DC52EF03CC595
:104E00002DF03BC52CF0030EFEEC00F02C0EEE6EE8
:104E1000020E016E42C52FF041C52EF040C52DF0A7
:104E20003FC52CF0030EFEEC00F02C0EEE6E020ED1
:104E3000016E46C52FF045C52EF044C52DF043C583
:104E40002CF0030EFEEC00F0EF6A72EC1CF01AEC92
:104E50001FF0140E24EC02F002EECAF0110EF76EF1
:104E6000760EF66ED9EC02F0020E016E086AEEC5FF
:104E700021F0EDC520F0CFEC00F02C0EEE6E020E0E
:104E8000016E086AF0C521F0EFC520F0CFEC00F00C
:104E90002C0EEE6E020E016E086AF2C521F0F1C50D
:104EA00020F0CFEC00F02C0EEE6E020E016E086AC0
:104EB000F4C521F0F3C520F0CFEC00F02C0EEE6E1F
:104EC000020E016E086AF6C521F0F5C520F0CFECA0
:104ED00000F02C0EEE6E020E016E086AF8C521F08D
:104EE000F7C520F0CFEC00F02C0EEE6E020E016E36
:104EF000086AFAC521F0F9C520F0CFEC00F02C0EBD
:104F0000EE6E020E016E000ECCEC00F02C0EEE6E7A
:104F1000020E016EE86A060109B9010ECCEC00F040
:104F2000EF6A000172EC1CF01AEC1FF0140E24EC76
:104F300002F002EECAF0110EF76E7E0EF66ED9EC9C
:104F400002F0020E016E086AFCC521F0FBC520F0DC
:104F5000CFEC00F02C0EEE6E020E016E086AFEC55C
:104F600021F0FDC520F0CFEC00F02C0EEE6E020E0D
:104F7000016E086A00C621F0FFC520F0CFEC00F0FA
:104F80002C0EEE6E020E016E086A02C621F001C6FA
:104F900020F0CFEC00F02C0EEE6E020E016E086ACF
:104FA00004C621F003C620F0CFEC00F02C0EEE6E0C
:104FB000020E016E086A06C621F005C620F0CFEC8D
:104FC00000F02C0EEE6E020E016E086A08C621F08B
:104FD00007C620F0CFEC00F02C0EEE6E020E016E34
:104FE000000ECCEC00F02C0EEE6E020E016EE86AA4
:104FF000060109BB010ECCEC00F0EF6A000172EC77
:105000001CF01AEC1FF0140E24EC02F002EECAF0B1
:10501000110EF76E860EF66ED9EC02F0020E016EDE
:105020000501E551CCEC00F02C0EEE6E020E016E87
:10503000086AD9C521F0D8C520F0CFEC00F02C0EBD
:10504000EE6E020E016E086ADBC521F0DAC520F0B3
:10505000CFEC00F0EF6A000172EC1CF01AEC1FF0CC
:10506000140E24EC02F0010E0401A35D0001D8A48B
:10507000C2EF29F002EECAF0110EF76E8E0EF66E38
:10508000D9EC02F0020E016EE86A82B8010ECCEC97
:1050900000F0020E016EE86A82BA010ECCEC00F05C
:1050A000020E016EE86A81B0010ECCEC00F0020E37
:1050B000016EE86A81B2010ECCEC00F0020E016EC6
:1050C000E86A81B4010ECCEC00F0300EEE6EEE6EAC
:1050D000EE6EEF6A72EC1CF01AEC1FF0140E24EC6A
:1050E00002F002EECAF0110EF76E960EF66ED9ECD3
:1050F00002F0020E016E3AC52FF039C52EF038C508
:105100002DF037C52CF0030EFEEC00F02C0EEE6EE9
:10511000020E016E3EC52FF03DC52EF03CC52DF0B0
:105120003BC52CF0030EFEEC00F02C0EEE6E020ED2
:10513000016E42C52FF041C52EF040C52DF03FC590
:105140002CF0030EFEEC00F02C0EEE6E020E016E43
:1051500046C52FF045C52EF044C52DF043C52CF0B3
:10516000030EFEEC00F0EF6A72EC1CF01AEC1FF07C
:10517000140E24EC02F002EECAF0110EF76E9E0E31
:10518000F66ED9EC02F0020E016E086AEEC521F04F
:10519000EDC520F0CFEC00F02C0EEE6E020E016E8D
:1051A000086AF0C521F0EFC520F0CFEC00F02C0E1E
:1051B000EE6E020E016E086AF2C521F0F1C520F014
:1051C000CFEC00F02C0EEE6E020E016E086AF4C5F4
:1051D00021F0F3C520F0CFEC00F02C0EEE6E020EA5
:1051E000016E086AF6C521F0F5C520F0CFEC00F09D
:1051F0002C0EEE6E020E016E086AF8C521F0F7C59E
:1052000020F0CFEC00F02C0EEE6E020E016E086A5C
:10521000FAC521F0F9C520F0CFEC00F02C0EEE6EAF
:10522000020E016E000ECCEC00F02C0EEE6E020EA3
:10523000016EE86A060109B9010ECCEC00F0EF6AD4
:10524000000172EC1CF01AEC1FF0140E24EC02F0BA
:1052500002EECAF0110EF76EA60EF66ED9EC02F051
:10526000020E016E086AFCC521F0FBC520F0CFECF0
:1052700000F02C0EEE6E020E016E086AFEC521F0E3
:10528000FDC520F0CFEC00F02C0EEE6E020E016E8C
:10529000086A00C621F0FFC520F0CFEC00F02C0E0C
:1052A000EE6E020E016E086A02C621F001C620F001
:1052B000CFEC00F02C0EEE6E020E016E086A04C6F2
:1052C00021F003C620F0CFEC00F02C0EEE6E020EA3
:1052D000016E086A06C621F005C620F0CFEC00F08A
:1052E0002C0EEE6E020E016E086A08C621F007C68B
:1052F00020F0CFEC00F02C0EEE6E020E016E000ED0
:10530000CCEC00F02C0EEE6E020E016EE86A060187
:1053100009BB010ECCEC00F0EF6A000172EC1CF04E
:105320001AEC1FF0140E24EC02F002EECAF0110E7B
:10533000F76EAE0EF66ED9EC02F0020E016E0501AC
:10534000E551CCEC00F02C0EEE6E020E016E086AF8
:10535000D9C521F0D8C520F0CFEC00F02C0EEE6EB0
:10536000020E016E086ADBC521F0DAC520F0CFEC31
:1053700000F0EF6A000172EC1CF01AEC1FF0140E42
:1053800024EC02F01200110EF76EB60EF66E01EE6E
:10539000DCF001EC03F0D8A4EAEF29F0010E0101E2
:1053A000CC6F0001040E0101CC5D0001D8B0E8EF24
:1053B00029F094928292FA0E24EC02F09492828266
:1053C000FA0E24EC02F00101CC2B0001D8A4E9D79D
:1053D00017EF2AF0010E0101CC6F0001030E01014D
:1053E000CC5D0001D8B017EF2AF094928292010EA2
:1053F0001D6EF40E25EC02F094928282C80E24EC0D
:1054000002F094928292010E1D6EF40E25EC02F0D1
:1054100094928282C80E24EC02F0010E1D6E900E52
:1054200025EC02F00101CC2B0001D8A4D6D7120044
:1054300001EEDCF0460EEE6E410EEE6E490EEE6EA3
:105440004C0EEE6EEF6A12008BEC2AF001EE31F09A
:10545000110EF76EBA0EF66ED9EC02F0020E016E66
:105460000501E551CCEC00F0110EF76ECE0EF66E94
:10547000D9EC02F0EF6A000161EC1CF0010E0101B1
:10548000CC6F0001040E0101CC5D0001D8B06EEFBD
:105490002AF094928292820E026E040E096E010E20
:1054A000046EF40E036E030E216EE80E206E33ECD4
:1054B00000F094928282820E026E040E096E010E3A
:1054C000046EF40E036E010E216E900E206E33EC0E
:1054D00000F00101CC2B0001D8A4D3D705EE92F047
:1054E000460EEE6E410EEE6E490EEE6E4C0EEE6EF8
:1054F000EF6A6FEC2BF094928292010E1D6EF40E07
:1055000025EC02F094928282010E1D6EF40E25ECC1
:1055100002F0F1D712008298829A81908192819450
:10552000120012000501256B01016B6B0601099742
:1055300000011200010E0501256F010E01016B6FC4
:105540000001120001EE31F084EC00F00501EB6F78
:1055500021C0ECF504EEA4F0110EF76EE00EF66E2D
:10556000D9EC02F0020E016E086AECC521F0EBC521
:1055700020F0CFEC00F0EF6A000125EC1EF01200E5
:10558000CADF2D0E0101CC6F010ED46F0001090E90
:105590000101D45D0001D8B012EF2BF094988288FD
:1055A0000101CC5124EC02F094988298949A828A5A
:1055B000CC5124EC02F0949A829A93908180CC5141
:1055C00024EC02F09390819093928182CC5124EC50
:1055D00002F09392819293948184CC5124EC02F056
:1055E0009394819493928182CC5124EC02F0939213
:1055F000819293908180CC5124EC02F09390819021
:10560000949A828ACC5124EC02F0949A829A9498CB
:105610008288CC5124EC02F094988298D42B00011B
:10562000D8A4B4D778DF120005EE92F011EE31F075
:10563000360EE75204E0E6CFEEFFE82EFAD7EF6A27
:105640006FEC2BF01200110EF76EFA0EF66E01EEF3
:1056500031F001EC03F0D8A43EEF2BF005012A85D0
:1056600004EEA4F0110EF76EFE0EF66ED9EC02F009
:10567000EF6A000125EC1EF04CEF2BF005012A9596
:1056800004EEA4F0120EF76E0C0EF66ED9EC02F0DA
:10569000EF6A000125EC1EF0120001EE31F084ECFF
:1056A00000F00501906F040E196EB00E186E1D6AA1
:1056B00090C51CF09CEC02F08E6F19C08FF504EEC3
:1056C000A4F0120EF76E1C0EF66ED9EC02F0020E6C
:1056D000016E9051CCEC00F0EF6A0001120004EE74
:1056E000A4F0120EF76E2E0EF66ED9EC02F015EE47
:1056F00092F0320EE75204E0E6CFEEFFE82EFAD742
:10570000EF6A25EC1EF0040E196EB00E186E1D6ABD
:1057100090C51CF09CEC02F005018E6F19C08FF54E
:105720009492828205EE92F0E86AEE5202E0E83E40
:10573000FCD7916F010E0101CC6F00010101CC512A
:105740000501915D0001D8A069EF2EF005EEC5F0CE
:1057500015EE92F0CCC1F3FF010EE1EC02F0EF6A1E
:10576000410E0501C55D0001D8A4C0EF2BF005EE88
:10577000CAF02E0EEE6E2D0EEE6EEF6A61EF2EF079
:10578000420E0501C55D0001D8A4D2EF2BF005EE55
:10579000CAF02D0EEE6E2E0EEE6EEE6EEE6EEF6A0F
:1057A00061EF2EF0430E0501C55D0001D8A4E6EFC0
:1057B0002BF005EECAF02D0EEE6E2E0EEE6E2D0EB7
:1057C000EE6E2E0EEE6EEF6A61EF2EF0440E0501C6
:1057D000C55D0001D8A4F7EF2BF005EECAF02D0E41
:1057E000EE6E2E0EEE6EEE6EEF6A61EF2EF0450E4F
:1057F0000501C55D0001D8A405EF2CF005EECAF047
:105800002E0EEE6EEF6A61EF2EF0460E0501C55DBD
:105810000001D8A418EF2CF005EECAF02E0EEE6EA3
:10582000EE6E2D0EEE6E2E0EEE6EEF6A61EF2EF026
:10583000470E0501C55D0001D8A429EF2CF005EE47
:10584000CAF02D0EEE6EEE6E2E0EEE6EEF6A61EF6A
:105850002EF0480E0501C55D0001D8A43AEF2CF0EA
:1058600005EECAF02E0EEE6EEE6EEE6EEE6EEF6A86
:1058700061EF2EF0490E0501C55D0001D8A449EF86
:105880002CF005EECAF02E0EEE6EEE6EEF6A61EFB2
:105890002EF04A0E0501C55D0001D8A45BEF2CF087
:1058A00005EECAF02E0EEE6E2D0EEE6EEE6EEE6E64
:1058B000EF6A61EF2EF04B0E0501C55D0001D8A423
:1058C0006DEF2CF005EECAF02D0EEE6E2E0EEE6E84
:1058D0002D0EEE6EEF6A61EF2EF04C0E0501C55DE8
:1058E0000001D8A480EF2CF005EECAF02E0EEE6E6B
:1058F0002D0EEE6E2E0EEE6EEE6EEF6A61EF2EF056
:105900004D0E0501C55D0001D8A48FEF2CF005EE0A
:10591000CAF02D0EEE6EEE6EEF6A61EF2EF04E0EB7
:105920000501C55D0001D8A49FEF2CF005EECAF07B
:105930002D0EEE6E2E0EEE6EEF6A61EF2EF04F0E14
:105940000501C55D0001D8A4AFEF2CF005EECAF04B
:105950002D0EEE6EEE6EEE6EEF6A61EF2EF0500ED3
:105960000501C55D0001D8A4C2EF2CF005EECAF018
:105970002E0EEE6E2D0EEE6EEE6E2E0EEE6EEF6AAB
:1059800061EF2EF0510E0501C55D0001D8A4D5EFE1
:105990002CF005EECAF02D0EEE6EEE6E2E0EEE6EB3
:1059A0002D0EEE6EEF6A61EF2EF0520E0501C55D11
:1059B0000001D8A4E7EF2CF005EECAF02E0EEE6E33
:1059C0002D0EEE6E2E0EEE6EEF6A61EF2EF0530E80
:1059D0000501C55D0001D8A4F7EF2CF005EECAF073
:1059E0002E0EEE6EEE6EEE6EEF6A61EF2EF0540E3E
:1059F0000501C55D0001D8A405EF2DF005EECAF044
:105A00002D0EEE6EEF6A61EF2EF0550E0501C55DAD
:105A10000001D8A416EF2DF005EECAF02E0EEE6EA2
:105A2000EE6E2D0EEE6EEF6A61EF2EF0560E050152
:105A3000C55D0001D8A428EF2DF005EECAF02E0EAA
:105A4000EE6EEE6EEE6E2D0EEE6EEF6A61EF2EF0E4
:105A5000570E0501C55D0001D8A439EF2DF005EE04
:105A6000CAF02E0EEE6E2D0EEE6EEE6EEF6A61EF48
:105A70002EF0580E0501C55D0001D8A44CEF2DF0A5
:105A800005EECAF02D0EEE6E2E0EEE6EEE6E2D0EA3
:105A9000EE6EEF6A61EF2EF0590E0501C55D000153
:105AA000D8A45FEF2DF005EECAF02D0EEE6E2E0E8F
:105AB000EE6E2D0EEE6EEE6EEF6A61EF2EF05A0E68
:105AC0000501C55D0001D8A471EF2DF005EECAF007
:105AD0002D0EEE6EEE6E2E0EEE6EEE6EEF6A61EF36
:105AE0002EF0300E0501C55D0001D8A483EF2DF026
:105AF00005EECAF02D0EEE6EEE6EEE6EEE6EEE6EF2
:105B0000EF6A61EF2EF0310E0501C55D0001D8A4EA
:105B100096EF2DF005EECAF02E0EEE6E2D0EEE6E07
:105B2000EE6EEE6EEE6EEF6A61EF2EF0320E050154
:105B3000C55D0001D8A4A9EF2DF005EECAF02E0E28
:105B4000EE6EEE6E2D0EEE6EEE6EEE6EEF6A61EFA5
:105B50002EF0330E0501C55D0001D8A4BCEF2DF079
:105B600005EECAF02E0EEE6EEE6EEE6E2D0EEE6EA1
:105B7000EE6EEF6A61EF2EF0340E0501C55D000197
:105B8000D8A4CEEF2DF005EECAF02E0EEE6EEE6E1E
:105B9000EE6E2D0EEE6EEF6A61EF2EF0350E050102
:105BA000C55D0001D8A4E0EF2DF005EECAF02E0E81
:105BB000EE6EEE6EEE6EEE6EEE6EEF6A61EF2EF052
:105BC000360E0501C55D0001D8A4F3EF2DF005EEFA
:105BD000CAF02D0EEE6E2E0EEE6EEE6EEE6EEE6EC8
:105BE000EF6A61EF2EF0370E0501C55D0001D8A404
:105BF00006EF2EF005EECAF02D0EEE6EEE6E2E0EB6
:105C0000EE6EEE6EEE6EEF6A61EF2EF0380E05016D
:105C1000C55D0001D8A419EF2EF005EECAF02D0ED7
:105C2000EE6EEE6EEE6E2E0EEE6EEE6EEF6A61EFC3
:105C30002EF0390E0501C55D0001D8A42CEF2EF021
:105C400005EECAF02D0EEE6EEE6EEE6EEE6E2E0EC0
:105C5000EE6EEF6A61EF2EF02F0E0501C55D0001BB
:105C6000D8A441EF2EF005EECAF02D0EEE6E2E0EEA
:105C7000EE6EEE6E2D0EEE6E2E0EEE6EEF6A61EF94
:105C80002EF03D0E0501C55D0001D8A455EF2EF0A4
:105C900005EECAF02D0EEE6E2E0EEE6EEE6EEE6E70
:105CA0002D0EEE6EEF6A61EF2EF0200E0501C55D40
:105CB0000001D8A461EF2EF005EECAF0200EEE6EC2
:105CC000EF6A6AEC2EF00101CC2B0001D8A49DEF05
:105CD0002BF0120005EECAF0E86AEE5202E0E83E50
:105CE000FCD70101D46F010ED76F00010101D7511C
:105CF000D45D0001D8A00BEF2FF005EEC7F015EE34
:105D0000CAF0D7C1F3FF010EE1EC02F0EF6A2E0EEC
:105D10000501C75D0001D8A4B6EF2EF094928292DF
:105D2000D89605012AA5D8860001D8B69AEF2EF09C
:105D300093948184820E026E040E096E8FC504F066
:105D40008EC503F08DC521F08CC520F033EC00F03A
:105D5000D89605012AA5D8860001D8B6B2EF2EF054
:105D6000939481949492828200EF2FF02D0E05017E
:105D7000C75D0001D8A4EBEF2EF094928292D896E2
:105D800005012AA5D8860001D8B6C9EF2EF0939454
:105D90008184820E026E040E096E05018F51030D7F
:105DA000F3CF04F08E51030DF3CF03F0F45004262B
:105DB0008DC521F08CC520F033EC00F0D8962AA5D3
:105DC000D8860001D8B6E7EF2EF093948194949290
:105DD000828200EF2FF0200E0501C75D0001D8A4DC
:105DE000FFEF2EF005018F51030DF3CF1DF08E5103
:105DF000030DF3CF1CF0F4501D2626EC02F0000139
:105E00008FC51DF005018E5125EC02F00101D72B45
:105E10000001D8A46AD705018F51030DF3CF1DF0FF
:105E20008E51030DF3CF1CF0F4501D2626EC02F02A
:105E300000011200000E0DEC02F005012F6F2DC0C5
:105E400030F5176A166A156A8F0E146E30C511F098
:105E50002FC510F0D0EC04F018EC04F013C0D2F110
:105E600012C0D1F111C0D0F110C0CFF1136A126A83
:105E7000200E116E810E106ED2C117F0D1C116F036
:105E8000D0C115F0CFC114F080EC04F013C02FF096
:105E900012C02EF011C02DF010C02CF02FC013F046
:105EA0002EC012F02DC011F02CC010F02EC517F02E
:105EB0002DC516F02CC515F02BC514F080EC04F0A0
:105EC00013C03AF512C039F511C038F510C037F5D6
:105ED0003AC513F039C512F038C511F037C510F0C6
:105EE0004AC517F049C516F048C515F047C514F066
:105EF0007EEC03F013C03AF512C039F511C038F545
:105F000010C037F5010E0DEC02F0316F2DC032F5E7
:105F1000176A166A156A8F0E146E32C511F031C5F4
:105F200010F0D0EC04F018EC04F013C0D2F112C061
:105F3000D1F111C0D0F110C0CFF1136A126A200E56
:105F4000116E810E106ED2C117F0D1C116F0D0C102
:105F500015F0CFC114F080EC04F013C02FF012C084
:105F60002EF011C02DF010C02CF02FC013F02EC059
:105F700012F02DC011F02CC010F02EC517F02DC559
:105F800016F02CC515F02BC514F080EC04F013C0EE
:105F90003EF512C03DF511C03CF510C03BF53EC5C5
:105FA00013F03DC512F03CC511F03BC510F04EC5D5
:105FB00017F04DC516F04CC515F04BC514F07EEC2E
:105FC00003F013C03EF512C03DF511C03CF510C002
:105FD0003BF5020E0DEC02F0336F2DC034F5176A5D
:105FE000166A156A8F0E146E34C511F033C510F0A1
:105FF000D0EC04F018EC04F013C0D2F112C0D1F1CF
:1060000011C0D0F110C0CFF1136A126A200E116EC8
:10601000810E106ED2C117F0D1C116F0D0C115F0AB
:10602000CFC114F080EC04F013C02FF012C02EF09A
:1060300011C02DF010C02CF02FC013F02EC012F0A4
:106040002DC011F02CC010F02EC517F02DC516F084
:106050002CC515F02BC514F080EC04F013C042F5EC
:1060600012C041F511C040F510C03FF542C513F014
:1060700041C512F040C511F03FC510F052C517F0F0
:1060800051C516F050C515F04FC514F07EEC03F065
:1060900013C042F512C041F511C040F510C03FF5E4
:1060A000030E0DEC02F0356F2DC036F5176A166A37
:1060B000156A8F0E146E36C511F035C510F0D0EC90
:1060C00004F018EC04F013C0D2F112C0D1F111C0E9
:1060D000D0F110C0CFF1136A126A200E116E810E3A
:1060E000106ED2C117F0D1C116F0D0C115F0CFC1DA
:1060F00014F080EC04F013C02FF012C02EF011C089
:106100002DF010C02CF02FC013F02EC012F02DC0B7
:1061100011F02CC010F02EC517F02DC516F02CC5AF
:1061200015F02BC514F080EC04F013C046F512C036
:1061300045F511C044F510C043F546C513F045C5FB
:1061400012F044C511F043C510F056C517F055C5FF
:1061500016F054C515F053C514F07EEC03F013C0CF
:1061600046F512C045F511C044F510C043F50001D5
:10617000120004EEA4F0120EF76E380EF66ED9EC93
:1061800002F0EF6A25EC1EF00A0E24EC02F052DE5B
:1061900004EEA4F0120EF76E5E0EF66ED9EC02F06D
:1061A000020E016E3AC52FF039C52EF038C52DF01C
:1061B00037C52CF0030EFEEC00F0120EF76E6E0EDB
:1061C000F66ED9EC02F0020E016E086A30C521F0BD
:1061D0002FC520F0CFEC00F0290EEE6EEF6A25EC13
:1061E0001EF004EEA4F0120EF76E780EF66ED9ECE7
:1061F00002F0020E016E3EC52FF03DC52EF03CC5EB
:106200002DF03BC52CF0030EFEEC00F0120EF76EE5
:10621000880EF66ED9EC02F0020E016E086A32C5E5
:1062200021F031C520F0CFEC00F0290EEE6EEF6AC0
:1062300025EC1EF004EEA4F0120EF76E920EF66E30
:10624000D9EC02F0020E016E42C52FF041C52EF0CE
:1062500040C52DF03FC52CF0030EFEEC00F0120EF1
:10626000F76EA20EF66ED9EC02F0020E016E086A0D
:1062700034C521F033C520F0CFEC00F0290EEE6ECE
:10628000EF6A25EC1EF004EEA4F0120EF76EAC0ED1
:10629000F66ED9EC02F0020E016E46C52FF045C530
:1062A0002EF044C52DF043C52CF0030EFEEC00F09B
:1062B000120EF76EBC0EF66ED9EC02F0020E016EF5
:1062C000086A36C521F035C520F0CFEC00F0290E64
:1062D000EE6EEF6A25EC1EF004EEA4F0120EF76EDF
:1062E000C60EF66ED9EC02F0EF6A25EC1EF00A0E2F
:1062F00024EC02F01200120EF76EEC0EF66E01EEB8
:1063000031F001EC03F0D8A495EF31F0010E01015A
:106310006C6F04EEA4F0120EF76EF00EF66ED9EC70
:1063200002F0EF6A000125EC1EF0130EF76E0C0E62
:10633000F66E01EE31F001EC03F0D8A4AEEF31F0CF
:1063400001016C6B04EEA4F0130EF76E100EF66EE6
:10635000D9EC02F0EF6A000125EC1EF012001200E9
:1063600001EE31F084EC00F020C010F021C011F0FB
:1063700022C012F023C013F0D2EC04F013C05AF57F
:1063800012C059F511C058F510C057F501EEA0F034
:10639000020E016E5AC52FF059C52EF058C52DF0CA
:1063A00057C52CF0030EFEEC00F0EF6A04EEA4F0EB
:1063B000130EF76E2C0EF66ED9EC02F011EEA0F073
:1063C000140EE75204E0E6CFEEFFE82EFAD7EF6AAC
:1063D00025EC1EF0120001EE31F084EC00F020C03C
:1063E00010F021C011F022C012F023C013F0D2EC43
:1063F00004F013C05EF512C05DF511C05CF510C06D
:106400005BF501EEA0F0020E016E5EC52FF05DC5DA
:106410002EF05CC52DF05BC52CF0030EFEEC00F0F9
:10642000EF6A04EEA4F0130EF76E420EF66ED9EC8E
:1064300002F011EEA0F0140EE75204E0E6CFEEFFFA
:10644000E82EFAD7EF6A25EC1EF0120001EE31F0CB
:1064500084EC00F020C010F021C011F022C012F036
:1064600023C013F0D2EC04F013C062F512C061F542
:1064700011C060F510C05FF501EEA0F0020E016ED4
:1064800062C52FF061C52EF060C52DF05FC52CF000
:10649000030EFEEC00F0EF6A04EEA4F0130EF76EAC
:1064A000580EF66ED9EC02F011EEA0F0140EE75281
:1064B00004E0E6CFEEFFE82EFAD7EF6A25EC1EF0F7
:1064C000120001EE31F084EC00F020C010F021C089
:1064D00011F022C012F023C013F0D2EC04F013C06C
:1064E00066F512C065F511C064F510C063F501EEE4
:1064F000A0F0020E016E66C52FF065C52EF064C5D2
:106500002DF063C52CF0030EFEEC00F0EF6A04EEF4
:10651000A4F0130EF76E6E0EF66ED9EC02F011EECB
:10652000A0F0140EE75204E0E6CFEEFFE82EFAD713
:10653000EF6A25EC1EF0120001EE31F084EC00F061
:1065400020C010F021C011F022C012F023C013F0BF
:10655000D2EC04F013C06AF512C069F511C068F5F9
:1065600010C067F501EEA0F0020E016E6AC52FF0B3
:1065700069C52EF068C52DF067C52CF0030EFEEC42
:1065800000F0EF6A04EEA4F0130EF76E840EF66EC0
:10659000D9EC02F011EEA0F0140EE75204E0E6CFC1
:1065A000EEFFE82EFAD7EF6A25EC1EF0120001EE9E
:1065B00031F084EC00F020C010F021C011F022C0B6
:1065C00012F023C013F0D2EC04F013C06EF512C029
:1065D0006DF511C06CF510C06BF501EEA0F0020E68
:1065E000016E6EC52FF06DC52EF06CC52DF06BC51C
:1065F0002CF0030EFEEC00F0EF6A04EEA4F0130E94
:10660000F76E9A0EF66ED9EC02F011EEA0F0140EB1
:10661000E75204E0E6CFEEFFE82EFAD7EF6A25EC6A
:106620001EF0120001EE31F084EC00F020C010F0FA
:1066300021C011F022C012F023C013F0D2EC04F0FC
:1066400013C072F512C071F511C070F510C06FF56E
:1066500001EEA0F0020E016E72C52FF071C52EF092
:1066600070C52DF06FC52CF0030EFEEC00F0EF6A44
:1066700004EEA4F0130EF76EB00EF66ED9EC02F035
:1066800011EEA0F0140EE75204E0E6CFEEFFE82E84
:10669000FAD7EF6A25EC1EF0120001EE31F084EC1F
:1066A00000F020C010F021C011F022C012F023C071
:1066B00013F0D2EC04F013C076F512C075F511C0DA
:1066C00074F510C073F501EEA0F0020E016E76C5F0
:1066D0002FF075C52EF074C52DF073C52CF0030E88
:1066E000FEEC00F0EF6A04EEA4F0130EF76EC60E97
:1066F000F66ED9EC02F011EEA0F0140EE75204E0B1
:10670000E6CFEEFFE82EFAD7EF6A25EC1EF0120076
:1067100001EE31F084EC00F020C010F021C011F047
:1067200022C012F023C013F0D2EC04F013C0D2F157
:1067300012C0D1F111C0D0F110C0CFF16F0E136EA5
:10674000120E126E030E116E750E106ED2C117F07E
:10675000D1C116F0D0C115F0CFC114F080EC04F017
:1067600013C04AF512C049F511C048F510C047F5ED
:1067700001EEA0F0020E016E4AC52FF049C52EF0C1
:1067800048C52DF047C52CF0030EFEEC00F0EF6A73
:1067900004EEA4F0130EF76EDC0EF66ED9EC02F0E8
:1067A00011EEA0F0140EE75204E0E6CFEEFFE82E63
:1067B000FAD7EF6A25EC1EF0120001EE31F084ECFE
:1067C00000F020C010F021C011F022C012F023C050
:1067D00013F0D2EC04F013C0D2F112C0D1F111C009
:1067E000D0F110C0CFF16F0E136E120E126E030EA9
:1067F000116E750E106ED2C117F0D1C116F0D0C156
:1068000015F0CFC114F080EC04F013C04EF512C0A7
:106810004DF511C04CF510C04BF501EEA0F0020E85
:10682000016E4EC52FF04DC52EF04CC52DF04BC559
:106830002CF0030EFEEC00F0EF6A04EEA4F0140E50
:10684000F76E020EF66ED9EC02F011EEA0F0140E07
:10685000E75204E0E6CFEEFFE82EFAD7EF6A25EC28
:106860001EF0120001EE31F084EC00F020C010F0B8
:1068700021C011F022C012F023C013F0D2EC04F0BA
:1068800013C0D2F112C0D1F111C0D0F110C0CFF1BC
:106890006F0E136E120E126E030E116E750E106EC9
:1068A000D2C117F0D1C116F0D0C115F0CFC114F08C
:1068B00080EC04F013C052F512C051F511C050F530
:1068C00010C04FF501EEA0F0020E016E52C52FF080
:1068D00051C52EF050C52DF04FC52CF0030EFEEC27
:1068E00000F0EF6A04EEA4F0140EF76E280EF66EB8
:1068F000D9EC02F011EEA0F0140EE75204E0E6CF5E
:10690000EEFFE82EFAD7EF6A25EC1EF0120001EE3A
:1069100031F084EC00F020C010F021C011F022C052
:1069200012F023C013F0D2EC04F013C0D2F112C065
:10693000D1F111C0D0F110C0CFF16F0E136E120E55
:10694000126E030E116E750E106ED2C117F0D1C10A
:1069500016F0D0C115F0CFC114F080EC04F013C0D4
:1069600056F512C055F511C054F510C053F501EE9F
:10697000A0F0020E016E56C52FF055C52EF054C57D
:106980002DF053C52CF0030EFEEC00F0EF6A04EE80
:10699000A4F0140EF76E4E0EF66ED9EC02F011EE66
:1069A000A0F0140EE75204E0E6CFEEFFE82EFAD78F
:1069B000EF6A25EC1EF012003AC513F039C512F04B
:1069C00038C511F037C510F05AC517F059C516F083
:1069D00058C515F057C514F00AEC03F00108D8B4F7
:1069E0000CEF35F09DEC35F06AC513F069C512F077
:1069F00068C511F067C510F03AC517F039C516F033
:106A000038C515F037C514F00AEC03F00108D8B406
:106A10000CEF35F069EC36F03EC513F03DC512F0D1
:106A20003CC511F03BC510F05EC517F05DC516F012
:106A30005CC515F05BC514F00AEC03F00108D8B48E
:106A40003CEF35F0D0EC35F06EC513F06DC512F0AB
:106A50006CC511F06BC510F03EC517F03DC516F0C2
:106A60003CC515F03BC514F00AEC03F00108D8B49E
:106A70003CEF35F09CEC36F042C513F041C512F006
:106A800040C511F03FC510F062C517F061C516F0A2
:106A900060C515F05FC514F00AEC03F00108D8B426
:106AA0006CEF35F003EC36F072C513F071C512F0DF
:106AB00070C511F06FC510F042C517F041C516F052
:106AC00040C515F03FC514F00AEC03F00108D8B436
:106AD0006CEF35F0CFEC36F046C513F045C512F03B
:106AE00044C511F043C510F066C517F065C516F032
:106AF00064C515F063C514F00AEC03F00108D8B4BE
:106B00009CEF35F036EC36F076C513F075C512F013
:106B100074C511F073C510F046C517F045C516F0E1
:106B200044C515F043C514F00AEC03F00108D8B4CD
:106B30009CEF35F002EC37F0120004EEA4F0140ED6
:106B4000F76E740EF66ED9EC02F0020E016E5AC5A5
:106B50002FF059C52EF058C52DF057C52CF0030E57
:106B6000FEEC00F0140EF76EA00EF66ED9EC02F0FB
:106B7000020E016E3AC52FF039C52EF038C52DF042
:106B800037C52CF0030EFEEC00F0760EEE6E2E0EE6
:106B9000EE6EEF6A25EC1EF0640E24EC02F012009B
:106BA00004EEA4F0140EF76EAE0EF66ED9EC02F001
:106BB000020E016E5EC52FF05DC52EF05CC52DF096
:106BC0005BC52CF0030EFEEC00F0140EF76EDA0E2F
:106BD000F66ED9EC02F0020E016E3EC52FF03DC5F7
:106BE0002EF03CC52DF03BC52CF0030EFEEC00F062
:106BF000760EEE6E2E0EEE6EEF6A25EC1EF0640E33
:106C000024EC02F0120004EEA4F0140EF76EE80E6D
:106C1000F66ED9EC02F0020E016E62C52FF061C56E
:106C20002EF060C52DF05FC52CF0030EFEEC00F0D9
:106C3000150EF76E140EF66ED9EC02F0020E016E10
:106C400042C52FF041C52EF040C52DF03FC52CF0B8
:106C5000030EFEEC00F0760EEE6E2E0EEE6EEF6A78
:106C600025EC1EF0640E24EC02F0120004EEA4F0F9
:106C7000150EF76E220EF66ED9EC02F0020E016EC2
:106C800066C52FF065C52EF064C52DF063C52CF0E8
:106C9000030EFEEC00F0150EF76E4E0EF66ED9ECFC
:106CA00002F0020E016E46C52FF045C52EF044C518
:106CB0002DF043C52CF0030EFEEC00F0760EEE6EC8
:106CC0002E0EEE6EEF6A25EC1EF0640E24EC02F040
:106CD000120004EEA4F0150EF76E5C0EF66ED9EC01
:106CE00002F0020E016E6AC52FF069C52EF068C56C
:106CF0002DF067C52CF0030EFEEC00F0150EF76EBC
:106D0000880EF66ED9EC02F0020E016E3AC52FF035
:106D100039C52EF038C52DF037C52CF0030EFEEC2A
:106D200000F0760EEE6E2E0EEE6EEF6A25EC1EF083
:106D3000640E24EC02F0120004EEA4F0150EF76EBF
:106D4000960EF66ED9EC02F0020E016E6EC52FF0B3
:106D50006DC52EF06CC52DF06BC52CF0030EFEEC4E
:106D600000F0150EF76EC20EF66ED9EC02F0020EB0
:106D7000016E3EC52FF03DC52EF03CC52DF03BC544
:106D80002CF0030EFEEC00F0760EEE6E2E0EEE6E84
:106D9000EF6A25EC1EF0640E24EC02F0120004EE03
:106DA000A4F0150EF76ED00EF66ED9EC02F0020EBE
:106DB000016E72C52FF071C52EF070C52DF06FC534
:106DC0002CF0030EFEEC00F0150EF76EFC0EF66EC6
:106DD000D9EC02F0020E016E42C52FF041C52EF033
:106DE00040C52DF03FC52CF0030EFEEC00F0760EF2
:106DF000EE6E2E0EEE6EEF6A25EC1EF0640E24ECA5
:106E000002F0120004EEA4F0160EF76E0A0EF66EF3
:106E1000D9EC02F0020E016E76C52FF075C52EF08A
:106E200074C52DF073C52CF0030EFEEC00F0160EA9
:106E3000F76E360EF66ED9EC02F0020E016E46C504
:106E40002FF045C52EF044C52DF043C52CF0030EA0
:106E5000FEEC00F0760EEE6E2E0EEE6EEF6A25EC76
:106E60001EF0640E24EC02F01200160EF76E440EB3
:106E7000F66E01EE31F001EC03F0D8A44EEF37F0DE
:106E80000501776B04EEA4F0160EF76E480EF66E51
:106E9000D9EC02F0EF6A000125EC1EF0160EF76E39
:106EA000680EF66E01EE31F001EC03F0D8A468EF45
:106EB00037F0010E0501776F04EEA4F0160EF76EA1
:106EC0006C0EF66ED9EC02F0EF6A000125EC1EF0B4
:106ED000160EF76E900EF66E01EE31F001EC03F037
:106EE000D8A482EF37F0020E0501776F04EEA4F00C
:106EF000160EF76E980EF66ED9EC02F0EF6A0001EE
:106F000025EC1EF01200010E0501775D0001D8A4EA
:106F1000A8EF37F03AC513F039C512F038C511F0B3
:106F200037C510F03EC517F03DC516F03CC515F04D
:106F30003BC514F042EC03F00108D8B4A5EF37F0DC
:106F4000060109830001A7EF37F00601099300014C
:106F5000020E0501775D0001D8A4E0EF37F03EC5D1
:106F600013F03DC512F03CC511F03BC510F07BC5D8
:106F700017F07AC516F079C515F078C514F00AEC4B
:106F800003F0356E3EC513F03DC512F03CC511F05F
:106F90003BC510F03AC517F039C516F038C515F0E5
:106FA00037C514F00AEC03F03510D8B4DDEF37F034
:106FB000060109830001DFEF37F0060109930001A4
:106FC000120001EE31F084EC00F020C010F021C07E
:106FD00011F022C012F023C013F0D2EC04F013C061
:106FE0007BF512C07AF511C079F510C078F5120062
:106FF000120001011B6B00019EAA01EF38F0AECF19
:107000001BF112009EB806EF38F0FCD71BC1ADFF94
:10701000120094928282D8960101D9A1D8860001EB
:10702000D8B61FEF38F0160EF76EC80EF66ED7EC16
:1070300001F00D0EDFEC01F00A0EDFEC01F0D89646
:10704000060109ABD8860001D8B672EF39F081A8E5
:107050002CEF38F09AEF3DF0E86A80BA010E356EF9
:10706000E86A81B6010E3510D8B439EF38F00EEF6A
:107070003CF0D8960501E6A9D8860001D8B65EEFA7
:1070800038F00101CE6B010ECD6F00010101CD5131
:107090000601035D0101CE51060104590001D8A08B
:1070A0005CEF38F0010E24EC02F00101CD2BD8B4D6
:1070B000CE2B0001D8A4E9D7939481940601015105
:1070C0000501EB5D060102510501EC590001D8B044
:1070D0006CEF38F02CEC26F081A871EF38F09AEFC5
:1070E0003DF0E86A80BA010E356EE86A81B6010E9D
:1070F0003510D8B47EEF38F0CCEF3BF0D8960501D0
:10710000E6ABD8860001D8B6A3EF38F00101CE6B0C
:10711000010ECD6F00010101CD510601015D01019C
:10712000CE51060102590001D8A0A1EF38F0010E9E
:1071300024EC02F00101CD2BD8B4CE2B0001D8A451
:10714000E9D7939281920501FF51EB5D0601005151
:107150000501EC590001D8B0B0EF38F02CEC26F066
:1071600081A8B5EF38F09AEF3DF0E86A80BA010ED9
:10717000356EE86A81B6010E3510D8B4C2EF38F02A
:107180008AEF3BF0D8960501E6ADD8860001D8B667
:10719000E7EF38F00101CE6B010ECD6F0001010168
:1071A000CD510501FF5D0101CE51060100590001DD
:1071B000D8A0E5EF38F0010E24EC02F00101CD2B50
:1071C000D8B4CE2B0001D8A4E9D7939081900501C3
:1071D000FD51EB5DFE51EC590001D8B0F2EF38F0F3
:1071E0002CEC26F081A8F7EF38F09AEF3DF0E86A32
:1071F00080BA010E356EE86A81B6010E3510D8B43A
:1072000004EF39F048EF3BF0D8960501E6AFD88699
:107210000001D8B629EF39F00101CE6B010ECD6F18
:1072200000010101CD510501FD5D0101CE510501B6
:10723000FE590001D8A027EF39F0010E24EC02F02E
:107240000101CD2BD8B4CE2B0001D8A4E9D7949A54
:10725000829A0501FB51EB5DFC51EC590001D8B05D
:1072600034EF39F02CEC26F081A839EF39F09AEFA1
:107270003DF0E86A80BA010E356EE86A81B6010E0B
:107280003510D8B446EF39F006EF3BF0D89606013A
:1072900009A1D8860001D8B66BEF39F00101CE6B99
:1072A000010ECD6F00010101CD510501FB5D010112
:1072B000CE510501FC590001D8A069EF39F0010E4B
:1072C00024EC02F00101CD2BD8B4CE2B0001D8A4C0
:1072D000E9D79498829881A870EF39F09AEF3DF041
:1072E000BEEF3AF081A877EF39F09AEF3DF0E86A07
:1072F00080BA010E356EE86A81B6010E3510D8B439
:1073000084EF39F053EF3DF0D8960501E6A9D88611
:107310000001D8B6A9EF39F00101CE6B010ECD6F97
:1073200000010101CD510501FB5D0101CE510501B7
:10733000FC590001D8A0A7EF39F0010E24EC02F0AF
:107340000101CD2BD8B4CE2B0001D8A4E9D7949855
:1073500082980501FD51EB5DFE51EC590001D8B05A
:10736000B4EF39F02CEC26F081A8B9EF39F09AEFA0
:107370003DF0E86A80BA010E356EE86A81B6010E0A
:107380003510D8B4C6EF39F011EF3DF0D8960501AD
:10739000E6ABD8860001D8B6EBEF39F00101CE6B31
:1073A000010ECD6F00010101CD510501FD5D01010F
:1073B000CE510501FE590001D8A0E9EF39F0010EC8
:1073C00024EC02F00101CD2BD8B4CE2B0001D8A4BF
:1073D000E9D7949A829A0501FF51EB5D06010051AD
:1073E0000501EC590001D8B0F8EF39F02CEC26F08B
:1073F00081A8FDEF39F09AEF3DF0E86A80BA010EFE
:10740000356EE86A81B6010E3510D8B40AEF3AF04D
:10741000CFEF3CF0D8960501E6ADD8860001D8B68E
:107420002FEF3AF00101CE6B010ECD6F000101018B
:10743000CD510501FF5D0101CE510601005900014A
:10744000D8A02DEF3AF0010E24EC02F00101CD2B73
:10745000D8B4CE2B0001D8A4E9D79390819006012F
:1074600001510501EB5D060102510501EC590001D6
:10747000D8B03DEF3AF02CEC26F081A842EF3AF07C
:107480009AEF3DF0E86A80BA010E356EE86A81B67F
:10749000010E3510D8B44FEF3AF08DEF3CF0D8968E
:1074A0000501E6AFD8860001D8B674EF3AF00101C5
:1074B000CE6B010ECD6F00010101CD510601015DC2
:1074C0000101CE51060102590001D8A072EF3AF035
:1074D000010E24EC02F00101CD2BD8B4CE2B00011B
:1074E000D8A4E9D793928192060103510501EB5D7F
:1074F000060104510501EC590001D8B082EF3AF0C1
:107500002CEC26F081A887EF3AF09AEF3DF0E86A7C
:1075100080BA010E356EE86A81B6010E3510D8B416
:1075200094EF3AF04BEF3CF0D896060109A1D886CB
:107530000001D8B6B9EF3AF00101CE6B010ECD6F64
:1075400000010101CD510601035D0101CE5106018B
:1075500004590001D8A0B7EF3AF0010E24EC02F074
:107560000101CD2BD8B4CE2B0001D8A4E9D7939438
:10757000819481A8BEEF3AF09AEF3DF005012A9D73
:10758000D896060109B7D8860001D8B6CAEF3AF0F6
:107590002CEC26F0EAEF17F0D896060109A3D8865E
:1075A0000001D8B6D6EF3AF0EAEF17F09492828253
:1075B000D8960101D9A1D8860001D8B6ECEF3AF0EF
:1075C000160EF76EE00EF66ED7EC01F00D0EDFEC46
:1075D00001F00A0EDFEC01F0D896060109A9D88661
:1075E0000001D8B63AEF3CF081A8F9EF3AF09AEFF3
:1075F0003DF0010E80BAE86A356E010E81B6E86A88
:107600003514D8B406EF3BF09AEF3DF0D89605015B
:10761000E6A9D8860001D8B62BEF3BF00101CE6B6E
:10762000010ECD6F00010101CD510501ED5D01019C
:10763000CE510501EE590001D8A029EF3BF0010E13
:1076400024EC02F00101CD2BD8B4CE2B0001D8A43C
:10765000E9D7949882880501EF51EB5DF051EC5920
:107660000001D8B036EF3BF02CEC26F081A83BEFC0
:107670003BF09AEF3DF0010E80BAE86A356E010EDC
:1076800081B6E86A3514D8B448EF3BF004EF39F01E
:10769000D8960501E6ABD8860001D8B66DEF3BF071
:1076A0000101CE6B010ECD6F00010101CD5105012D
:1076B000EF5D0101CE510501F0590001D8A06BEF3B
:1076C0003BF0010E24EC02F00101CD2BD8B4CE2BFF
:1076D0000001D8A4E9D7949A828A0501F151EB5DA3
:1076E000F251EC590001D8B078EF3BF02CEC26F0C9
:1076F00081A87DEF3BF09AEF3DF0010E80BAE86A79
:10770000356E010E81B6E86A3514D8B48AEF3BF0C5
:10771000C2EF38F0D8960501E6ADD8860001D8B69C
:10772000AFEF3BF00101CE6B010ECD6F0001010107
:10773000CD510501F15D0101CE510501F259000164
:10774000D8A0ADEF3BF0010E24EC02F00101CD2BEF
:10775000D8B4CE2B0001D8A4E9D79390818005013D
:10776000F351EB5DF451EC590001D8B0BAEF3BF0A6
:107770002CEC26F081A8BFEF3BF09AEF3DF0010E14
:1077800080BAE86A356E010E81B6E86A3514D8B45D
:10779000CCEF3BF07EEF38F0D8960501E6AFD88607
:1077A0000001D8B6F1EF3BF00101CE6B010ECD6FB9
:1077B00000010101CD510501F35D0101CE5105012B
:1077C000F4590001D8A0EFEF3BF0010E24EC02F0D9
:1077D0000101CD2BD8B4CE2B0001D8A4E9D79392C8
:1077E00081820501F551EB5DF651EC590001D8B0ED
:1077F000FCEF3BF02CEC26F081A801EF3CF09AEF77
:107800003DF0010E80BAE86A356E010E81B6E86A75
:107810003514D8B40EEF3CF039EF38F0D8960601A5
:1078200009A1D8860001D8B633EF3CF00101CE6B38
:10783000010ECD6F00010101CD510501F55D010182
:10784000CE510501F6590001D8A031EF3CF0010EF0
:1078500024EC02F00101CD2BD8B4CE2B0001D8A42A
:10786000E9D79394818481A838EF3CF09AEF3DF0FA
:107870007DEF3DF081A83FEF3CF09AEF3DF0010E27
:1078800080BAE86A356E010E81B6E86A3514D8B45C
:107890004BEF3CF049D6D8960501E6A9D886000101
:1078A000D8B670EF3CF00101CE6B010ECD6F000138
:1078B0000101CD510501F55D0101CE510501F659DA
:1078C0000001D8A06EEF3CF0010E24EC02F00101A3
:1078D000CD2BD8B4CE2B0001D8A4E9D793948184C2
:1078E0000501F351EB5DF451EC590001D8B07BEF89
:1078F0003CF02CEC26F081A880EF3CF09AEF3DF0B4
:10790000010E80BAE86A356E010E81B6E86A351458
:10791000D8B48DEF3CF04FEF3AF0D8960501E6ABC6
:10792000D8860001D8B6B2EF3CF00101CE6B010E53
:10793000CD6F00010101CD510501F35D0101CE5173
:107940000501F4590001D8A0B0EF3CF0010E24EC81
:1079500002F00101CD2BD8B4CE2B0001D8A4E9D779
:10796000939281820501F151EB5DF251EC590001D6
:10797000D8B0BDEF3CF02CEC26F081A8C2EF3CF073
:107980009AEF3DF0010E80BAE86A356E010E81B6BD
:10799000E86A3514D8B4CFEF3CF00AEF3AF0D89645
:1079A0000501E6ADD8860001D8B6F4EF3CF0010140
:1079B000CE6B010ECD6F00010101CD510501F15DCE
:1079C0000101CE510501F2590001D8A0F2EF3CF0BF
:1079D000010E24EC02F00101CD2BD8B4CE2B000116
:1079E000D8A4E9D7939081800501EF51EB5DF05168
:1079F000EC590001D8B0FFEF3CF02CEC26F081A848
:107A000004EF3DF09AEF3DF0010E80BAE86A356E62
:107A1000010E81B6E86A3514D8B411EF3DF0C6EF17
:107A200039F0D8960501E6AFD8860001D8B636EF12
:107A30003DF00101CE6B010ECD6F00010101CD5172
:107A40000501EF5D0101CE510501F0590001D8A0FB
:107A500034EF3DF0010E24EC02F00101CD2BD8B43F
:107A6000CE2B0001D8A4E9D7949A828A0501ED5162
:107A7000EB5DEE51EC590001D8B041EF3DF02CEC3C
:107A800026F081A846EF3DF09AEF3DF0010E80BA56
:107A9000E86A356E010E81B6E86A3514D8B453EF42
:107AA0003DF084EF39F0D896060109A1D88600018F
:107AB000D8B678EF3DF00101CE6B010ECD6F00011D
:107AC0000101CD510501ED5D0101CE510501EE59D8
:107AD0000001D8A076EF3DF0010E24EC02F0010188
:107AE000CD2BD8B4CE2B0001D8A4E9D794988288A6
:107AF00081A87DEF3DF09AEF3DF005012A8DD896E3
:107B0000060109B7D8860001D8B689EF3DF02CEC04
:107B100026F0EAEF17F005012A9D0001EAEF17F0C1
:107B200005012A8D000181A898EF3DF09AEF3DF004
:107B3000EAEF17F08BEC2AF0EAEF17F0160EF76E6B
:107B4000F60EF66E01EE31F001EC03F0D8A4ACEFC6
:107B50003DF0010E01016B6F0001160EF76EFE0E77
:107B6000F66E01EE31F001EC03F0D8A4C6EF3DF063
:107B700001016B6B04EEA4F0170EF76E060EF66EA5
:107B8000D9EC02F0EF6A000125EC1EF01200170E8E
:107B9000F76E1C0EF66E01EE31F001EC03F0D8A486
:107BA000DAEF3DF006010987010E0101686F00015F
:107BB000EAEF3DF0060109970101686B04EEA4F0BD
:107BC000170EF76E200EF66ED9EC02F0EF6A000188
:107BD00025EC1EF01200170EF76E300EF66E01EE59
:107BE00031F001EC03F0D8A4FBEF3DF0060109975A
:107BF0000101686B696B0001170EF76E360EF66EA9
:107C000001EE31F001EC03F0D8A40EEF3EF00601D6
:107C10000987010E0101686F010E696F00011200F2
:107C200005EED0F011EE31F0060EE6CFEEFFE82EB5
:107C3000FCD7EF6A04EEA4F0170EF76E3E0EF66E58
:107C4000D9EC02F015EED0F0060EE75204E0E6CFD4
:107C5000EEFFE82EFAD7EF6A25EC1EF0120005EED3
:107C600092F015EED0F0060EE75204E0E6CFEEFFFC
:107C7000E82EFAD7EF6A6FEC2BF0120004EEA4F0B6
:107C8000170EF76E500EF66ED9EC02F011EE31F0D1
:107C9000360EE75204E0E6CFEEFFE82EFAD7EF6AA1
:107CA00025EC1EF001EE31F084EC00F00501D86FF8
:107CB00021C0D9F50001120004EEA4F0170EF76EF2
:107CC000660EF66ED9EC02F011EE31F0360EE75288
:107CD00004E0E6CFEEFFE82EFAD7EF6A25EC1EF0BF
:107CE00001EE31F084EC00F00501DA6F21C0DBF524
:107CF00000011200F8EC37F004EEA4F0170EF76E56
:107D00007E0EF66ED9EC02F0020E016E0501E55111
:107D1000CCEC00F0EF6A000125EC1EF0120004EE3E
:107D2000A4F0170EF76E960EF66ED9EC02F011EE77
:107D300031F0360EE75204E0E6CFEEFFE82EFAD738
:107D40002E0EEE6EEF6A25EC1EF001EE31F084ECA3
:107D500000F00501E56F0001120004EEA4F0170E1B
:107D6000F76EB20EF66ED9EC02F011EE31F0360E6F
:107D7000E75204E0E6CFEEFFE82EFAD7200EEE6ED3
:107D80006D0EEE6E730EEE6E2E0EEE6EEF6A25EC3D
:107D90001EF001EE31F084EC00F00501ED6F21C022
:107DA000EEF50001120004EEA4F0170EF76EC80EF7
:107DB000F66ED9EC02F011EE31F0360EE75204E027
:107DC000E6CFEEFFE82EFAD7200EEE6E6D0EEE6EC9
:107DD000730EEE6E2E0EEE6EEF6A25EC1EF001EEC7
:107DE00031F084EC00F00501EF6F21C0F0F50001E7
:107DF000120004EEA4F0170EF76EDE0EF66ED9EC4C
:107E000002F011EE31F0360EE75204E0E6CFEEFF5D
:107E1000E82EFAD7200EEE6E6D0EEE6E730EEE6E3D
:107E20002E0EEE6EEF6A25EC1EF001EE31F084ECC2
:107E300000F00501F16F21C0F2F50001120004EE1F
:107E4000A4F0170EF76EF40EF66ED9EC02F011EEF8
:107E500031F0360EE75204E0E6CFEEFFE82EFAD717
:107E6000200EEE6E6D0EEE6E730EEE6E2E0EEE6E3C
:107E7000EF6A25EC1EF001EE31F084EC00F0050114
:107E8000F36F21C0F4F50001120004EEA4F0180E07
:107E9000F76E0A0EF66ED9EC02F011EE31F0360EE6
:107EA000E75204E0E6CFEEFFE82EFAD7200EEE6EA2
:107EB0006D0EEE6E730EEE6E2E0EEE6EEF6A25EC0C
:107EC0001EF001EE31F084EC00F00501F56F21C0E9
:107ED000F6F50001120004EEA4F0180EF76E200E65
:107EE000F66ED9EC02F011EE31F0360EE75204E0F6
:107EF000E6CFEEFFE82EFAD7200EEE6E6D0EEE6E98
:107F0000730EEE6E2E0EEE6EEF6A25EC1EF001EE95
:107F100031F084EC00F00501FB6F21C0FCF500019D
:107F2000120004EEA4F0180EF76E340EF66ED9ECC3
:107F300002F011EE31F0360EE75204E0E6CFEEFF2C
:107F4000E82EFAD7200EEE6E6D0EEE6E730EEE6E0C
:107F50002E0EEE6EEF6A25EC1EF001EE31F084EC91
:107F600000F00501FD6F21C0FEF50001120004EED6
:107F7000A4F0180EF76E480EF66ED9EC02F011EE72
:107F800031F0360EE75204E0E6CFEEFFE82EFAD7E6
:107F9000200EEE6E6D0EEE6E730EEE6E2E0EEE6E0B
:107FA000EF6A25EC1EF001EE31F084EC00F00501E3
:107FB000FF6F21C000F60001120004EEA4F0180EBD
:107FC000F76E5C0EF66ED9EC02F011EE31F0360E63
:107FD000E75204E0E6CFEEFFE82EFAD7200EEE6E71
:107FE0006D0EEE6E730EEE6E2E0EEE6EEF6A25ECDB
:107FF0001EF001EE31F084EC00F00601016F21C0AB
:1080000002F60001120004EEA4F0180EF76E700ED6
:10801000F66ED9EC02F011EE31F0360EE75204E0C4
:10802000E6CFEEFFE82EFAD7200EEE6E6D0EEE6E66
:10803000730EEE6E2E0EEE6EEF6A25EC1EF001EE64
:1080400031F084EC00F00601036F21C004F600015A
:108050001200310E0101315D0001D8A437EF40F06C
:108060000501E68901EEA0F0310EEE6EEF6A000127
:10807000320E0101315D0001D8A446EF40F0050148
:10808000E68B01EEA0F0320EEE6EEF6A0001330EC9
:108090000101315D0001D8A455EF40F00501E68DE6
:1080A00001EEA0F0330EEE6EEF6A0001340E010116
:1080B000315D0001D8A464EF40F00501E68F01EEC8
:1080C000A0F0340EEE6EEF6A0001350E0101315D55
:1080D0000001D8A473EF40F00601098101EEA0F081
:1080E000350EEE6EEF6A000104EEA4F0180EF76E86
:1080F000840EF66ED9EC02F011EEA0F0140EE752E9
:1081000004E0E6CFEEFFE82EFAD7180EF76E8C0EDD
:10811000F66ED9EC02F0EF6A25EC1EF01200310E7B
:108120000101315D0001D8A49DEF40F00501E69901
:1081300001EEA0F0310EEE6EEF6A0001320E010189
:10814000315D0001D8A4ACEF40F00501E69B01EEE3
:10815000A0F0320EEE6EEF6A0001330E0101315DC8
:108160000001D8A4BBEF40F00501E69D01EEA0F0B0
:10817000330EEE6EEF6A0001340E0101315D000135
:10818000D8A4CAEF40F00501E69F01EEA0F0340E3E
:10819000EE6EEF6A0001350E0101315D0001D8A4D9
:1081A000D9EF40F00601099101EEA0F0350EEE6E18
:1081B000EF6A000104EEA4F0180EF76E960EF66E4C
:1081C000D9EC02F011EEA0F0140EE75204E0E6CF75
:1081D000EEFFE82EFAD7180EF76E9E0EF66ED9EC6B
:1081E00002F0EF6A25EC1EF01200180EF76EA80ED2
:1081F000F66E01EE31F001EC03F0D8A401EF41F08E
:108200008288180EF76EAC0EF66E01EE31F001ECBE
:1082100003F0D8A40DEF41F0829882A81BEF41F043
:1082200004EEA4F0180EF76EB00EF66ED9EC02F064
:10823000EF6A25EC1EF082B829EF41F004EEA4F0BD
:10824000180EF76EC20EF66ED9EC02F0EF6A25EC4E
:108250001EF01200180EF76ED40EF66E01EE31F01D
:1082600001EC03F0D8A436EF41F0828A180EF76EC5
:10827000D80EF66E01EE31F001EC03F0D8A442EF17
:1082800041F0829A82AA50EF41F004EEA4F0180E59
:10829000F76EDC0EF66ED9EC02F0EF6A25EC1EF0FC
:1082A00082BA5EEF41F004EEA4F0180EF76EEE0E07
:1082B000F66ED9EC02F0EF6A25EC1EF01200190EF2
:1082C000F76E000EF66E01EE31F001EC03F0D8A46B
:1082D0006BEF41F08180190EF76E040EF66E01EE21
:1082E00031F001EC03F0D8A477EF41F0819081A048
:1082F00085EF41F004EEA4F0190EF76E080EF66E4D
:10830000D9EC02F0EF6A25EC1EF081B093EF41F05A
:1083100004EEA4F0190EF76E1A0EF66ED9EC02F008
:10832000EF6A25EC1EF01200190EF76E2C0EF66E99
:1083300001EE31F001EC03F0D8A4A0EF41F081820E
:10834000190EF76E300EF66E01EE31F001EC03F00F
:10835000D8A4ACEF41F0819281A2BAEF41F004EED3
:10836000A4F0190EF76E340EF66ED9EC02F0EF6A37
:1083700025EC1EF081B2C8EF41F004EEA4F0190E16
:10838000F76E460EF66ED9EC02F0EF6A25EC1EF0A1
:108390001200190EF76E580EF66E01EE31F001EC78
:1083A00003F0D8A4D5EF41F08184190EF76E5C0E6E
:1083B000F66E01EE31F001EC03F0D8A4E1EF41F0EC
:1083C000819481A4EFEF41F004EEA4F0190EF76E52
:1083D000600EF66ED9EC02F0EF6A25EC1EF081B467
:1083E000FDEF41F004EEA4F0190EF76E720EF66E7A
:1083F000D9EC02F0EF6A25EC1EF012001200120018
:108400001200190EF76E840EF66E01EE31F001ECDB
:1084100003F0D8A40EEF42F006010B8F0001190EF5
:10842000F76E880EF66E01EE31F001EC03F0D8A481
:108430001CEF42F006010B9F0001D89606010BAF1E
:10844000D8860001D8B630EF42F004EEA4F0190E41
:10845000F76E8C0EF66ED9EC02F0EF6A25EC1EF08A
:10846000D89606010BBFD8860001D8B643EF42F07C
:1084700004EEA4F0190EF76E9C0EF66ED9EC02F025
:10848000EF6A25EC1EF00601098D00011200190E9D
:10849000F76EAE0EF66E01EE31F001EC03F0D8A4EB
:1084A00054EF42F006010C810001190EF76EB20E76
:1084B000F66E01EE31F001EC03F0D8A462EF42F069
:1084C00006010C910001D89606010CA1D886000186
:1084D000D8B676EF42F004EEA4F0190EF76EB60EA1
:1084E000F66ED9EC02F0EF6A25EC1EF0D896060184
:1084F0000CB1D8860001D8B689EF42F004EEA4F0A2
:10850000190EF76EC60EF66ED9EC02F0EF6A25EC86
:108510001EF00601098D00011200190EF76ED80E2B
:10852000F66E01EE31F001EC03F0D8A49AEF42F0C0
:1085300006010C830001190EF76EDC0EF66E01EEDB
:1085400031F001EC03F0D8A4A8EF42F006010C933F
:108550000001D89606010CA3D8860001D8B6BCEF5E
:1085600042F004EEA4F0190EF76EE00EF66ED9ECB0
:1085700002F0EF6A25EC1EF0D89606010CB3D886FF
:108580000001D8B6CFEF42F004EEA4F0190EF76E5A
:10859000F00EF66ED9EC02F0EF6A25EC1EF0060143
:1085A000098D0001120004EEA4F01A0EF76E020EFF
:1085B000F66ED9EC02F0EF6A25EC1EF0010E050113
:1085C000E56F010EE36FEE6B010EED6FF06B640E65
:1085D000EF6FF26B640EF16FF46B640EF36FF66B7A
:1085E000640EF56FF86B640EF76FFA6B640EF96F3B
:1085F000FC6B010EFB6FFE6B640EFD6F0601006BE2
:10860000640E0501FF6F0601026B640E016F046BBF
:10861000640E036F066B640E056F086B640E076FC4
:108620000989098B140E0501906F776BCD0E7B6F56
:10863000CC0E7A6F4C0E796F7C0E786F060109951F
:1086400005014A6B496B486B476B4E6B4D6B4C6B2E
:108650004B6B526B516B506B4F6B566B556B546B36
:10866000536B010169530001D8A439EF43F05BEC6F
:108670004AF001016B6B686B060109970501256BD8
:108680005A6B596B586B576B5E6B5D6B5C6B5B6BBE
:10869000626B616B606B5F6B666B656B646B636B6E
:1086A0006A6B696B700E686F830E676F6E6B6D6BB4
:1086B000700E6C6F830E6B6F726B716B700E706FE0
:1086C000830E6F6F766B756B700E746F830E736FA6
:1086D0000401A36B01016C6B0501EC6BFA0EEB6FEF
:1086E00000011200010E0501D76FAA6AA96AD751CD
:1086F000FEEC01F00A0E24EC02F0AA6A020EA96E4A
:10870000D851FEEC01F0D951FEEC01F00A0E24EC38
:1087100002F0AA6A040EA96EDA51FEEC01F0DB51F8
:10872000FEEC01F00A0E24EC02F0AA6A060EA96E15
:10873000E551FEEC01F00A0E24EC02F0AA6A0A0EE2
:10874000A96E000EFEEC01F0AA6A140EA96EED519E
:10875000FEEC01F0EE51FEEC01F00A0E24EC02F00A
:10876000AA6A160EA96EEF51FEEC01F0F051FEEC74
:1087700001F00A0E24EC02F0AA6A180EA96EF1515B
:10878000FEEC01F0F251FEEC01F00A0E24EC02F0D6
:10879000AA6A1A0EA96EF351FEEC01F0F451FEEC38
:1087A00001F00A0E24EC02F0AA6A1C0EA96EF55123
:1087B000FEEC01F0F651FEEC01F00A0E24EC02F0A2
:1087C000AA6A1E0EA96EF751FEEC01F0F851FEECFC
:1087D00001F00A0E24EC02F0AA6A200EA96EF951EB
:1087E000FEEC01F0FA51FEEC01F00A0E24EC02F06E
:1087F000AA6A280EA96EFB51FEEC01F0FC51FEECBA
:1088000001F00A0E24EC02F0AA6A2A0EA96EFD51AC
:10881000FEEC01F0FE51FEEC01F00A0E24EC02F039
:10882000AA6A2C0EA96EFF51FEEC01F00601005160
:10883000FEEC01F00A0E24EC02F0AA6A2E0EA96EDC
:108840000151FEEC01F00251FEEC01F00A0E24ECA5
:1088500002F0AA6A300EA96E0351FEEC01F0045139
:10886000FEEC01F00A0E24EC02F0AA6A320EA96EA8
:108870000551FEEC01F00651FEEC01F00A0E24EC6D
:1088800002F0AA6A340EA96E0751FEEC01F00851FD
:10889000FEEC01F00A0E24EC02F0AA6A3C0EA96E6E
:1088A000E86A09B9010EFEEC01F00A0E24EC02F0B0
:1088B000AA6A3E0EA96EE86A09BB010EFEEC01F041
:1088C0000A0E24EC02F0AA6A400EA96E0401A3511C
:1088D000FEEC01F00A0E24EC02F0AA6A410EA96E29
:1088E00005EED0F0EE5003E0FEEC01F0FBD70A0EEF
:1088F00024EC02F001EECAF015EED0F0010EF36E9A
:10890000010EE1EC02F0EF6AAA6A410EA96E01EED7
:10891000CAF0EE5003E0FEEC01F0FBD70A0E24ECA7
:1089200002F001EECAF015EED0F0020EF36E010E69
:10893000E1EC02F0EF6AAA6A420EA96E01EECAF0FB
:10894000EE5003E0FEEC01F0FBD70A0E24EC02F03F
:1089500001EECAF015EED0F0030EF36E010EE1EC5D
:1089600002F0EF6AAA6A430EA96E01EECAF0EE5059
:1089700003E0FEEC01F0FBD70A0E24EC02F001EE5E
:10898000CAF015EED0F0040EF36E010EE1EC02F029
:10899000EF6AAA6A440EA96E01EECAF0EE5003E037
:1089A000FEEC01F0FBD70A0E24EC02F001EECAF057
:1089B00015EED0F0050EF36E010EE1EC02F0EF6A59
:1089C000AA6A450EA96E01EECAF0EE5003E0FEEC75
:1089D00001F0FBD70A0E24EC02F001EECAF015EE0E
:1089E000D0F0060EF36E010EE1EC02F0EF6AAA6A17
:1089F000460EA96E01EECAF0EE5003E0FEEC01F067
:108A0000FBD70A0E24EC02F0AA6A500EA96EE86A9F
:108A10000501E6B9010EFEEC01F00A0E24EC02F0AD
:108A2000AA6A510EA96EE86AE6BB010EFEEC01F0DF
:108A30000A0E24EC02F0AA6A520EA96EE86AE6BD9C
:108A4000010EFEEC01F00A0E24EC02F0AA6A530EAD
:108A5000A96EE86AE6BF010EFEEC01F00A0E24ECF6
:108A600002F0AA6A540EA96EE86A060109B1010E65
:108A7000FEEC01F00A0E24EC02F0AA6A550EA96E73
:108A800005019051FEEC01F00A0E24EC02F0AA6AF6
:108A9000560EA96E7751FEEC01F00A0E24EC02F09E
:108AA000AA6A570EA96E7851FEEC01F07951FEECDE
:108AB00001F07A51FEEC01F07B51FEEC01F00A0E60
:108AC00024EC02F0AA6A5B0EA96EE86A060109B7F7
:108AD000010EFEEC01F00A0E24EC02F0AA6A5C0E14
:108AE000A96E05014751FEEC01F04851FEEC01F082
:108AF0004951FEEC01F04A51FEEC01F00A0E24EC63
:108B000002F0AA6A600EA96E4B51FEEC01F04C51C6
:108B1000FEEC01F04D51FEEC01F04E51FEEC01F087
:108B20000A0E24EC02F0AA6A640EA96E4F51FEEC04
:108B300001F05051FEEC01F05151FEEC01F05251A8
:108B4000FEEC01F00A0E24EC02F0AA6A680EA96E8F
:108B50005351FEEC01F05451FEEC01F05551FEEC86
:108B600001F05651FEEC01F00A0E24EC02F0AA6A64
:108B70006C0EA96E01016851FEEC01F00A0E24ECA6
:108B800002F0AA6A6D0EA96E6951FEEC01F00A0EA0
:108B900024EC02F0AA6A6E0EA96E6B51FEEC01F095
:108BA0000A0E24EC02F0AA6A6F0EA96E0501575155
:108BB000FEEC01F05851FEEC01F05951FEEC01F0D1
:108BC0005A51FEEC01F00A0E24EC02F0AA6A730E70
:108BD000A96E5B51FEEC01F05C51FEEC01F05D51C1
:108BE000FEEC01F05E51FEEC01F00A0E24EC02F006
:108BF000AA6A770EA96E5F51FEEC01F06051FEEC9F
:108C000001F06151FEEC01F06251FEEC01F00A0E40
:108C100024EC02F0AA6A7B0EA96E6351FEEC01F00F
:108C20006451FEEC01F06551FEEC01F06651FEEC82
:108C300001F00A0E24EC02F0AA6A7F0EA96E6751B9
:108C4000FEEC01F06851FEEC01F06951FEEC01F020
:108C50006A51FEEC01F00A0E24EC02F0AA6A830EBF
:108C6000A96E6B51FEEC01F06C51FEEC01F06D5100
:108C7000FEEC01F06E51FEEC01F00A0E24EC02F065
:108C8000AA6A870EA96E6F51FEEC01F07051FEECDE
:108C900001F07151FEEC01F07251FEEC01F00A0E90
:108CA00024EC02F0AA6A8B0EA96E7351FEEC01F05F
:108CB0007451FEEC01F07551FEEC01F07651FEECC2
:108CC00001F00A0E24EC02F0AA6A8F0EA96E0101CF
:108CD0006C51FEEC01F00A0E24EC02F0AA6A900E30
:108CE000A96E05012551FEEC01F00A0E24EC02F0FC
:108CF000AA6A910EA96EEB51FEEC01F0EC51FEEC6C
:108D000001F00A0E24EC02F004EEA4F01A0EF76E45
:108D10002A0EF66ED9EC02F0EF6A000125EC1EF087
:108D20001200000EF5EC01F00501D76F020EF5EC14
:108D300001F0D86FF7EC01F0D96F040EF5EC01F0FB
:108D4000DA6FF7EC01F0DB6F060EF5EC01F0E56F82
:108D50000A0EF5EC01F0E36FE329E46F140EF5EC75
:108D600001F0ED6FF7EC01F0EE6F160EF5EC01F08F
:108D7000EF6FF7EC01F0F06F180EF5EC01F0F16F0A
:108D8000F7EC01F0F26F1A0EF5EC01F0F36FF7EC6F
:108D900001F0F46F1C0EF5EC01F0F56FF7EC01F04B
:108DA000F66F1E0EF5EC01F0F76FF7EC01F0F86FBF
:108DB000200EF5EC01F0F96FF7EC01F0FA6F280ED8
:108DC000F5EC01F0FB6FF7EC01F0FC6F2A0EF5EC0F
:108DD00001F0FD6FF7EC01F0FE6F2C0EF5EC01F0E9
:108DE000FF6FF7EC01F00601006F2E0EF5EC01F0BD
:108DF000016FF7EC01F0026F300EF5EC01F0036F3C
:108E0000F7EC01F0046F320EF5EC01F0056FF7ECB2
:108E100001F0066F340EF5EC01F0076FF7EC01F08E
:108E2000086F3C0EF5EC01F00989E8A009993E0EA7
:108E3000F5EC01F0098BE8A0099B400EF5EC01F080
:108E40000401A36F500EF5EC01F00501E689E8A0DE
:108E5000E699510EF5EC01F0E68BE8A0E69B520E88
:108E6000F5EC01F0E68DE8A0E69D530EF5EC01F07F
:108E7000E68FE8A0E69F540EF5EC01F006010981AB
:108E8000E8A00991550EF5EC01F00501906F560E22
:108E9000F5EC01F0776F570EF5EC01F0786FF7EC19
:108EA00001F0796FF7EC01F07A6FF7EC01F07B6F6E
:108EB0005B0EF5EC01F006010987E8A009975C0E4E
:108EC000F5EC01F00501476FF7EC01F0486FF7ECA6
:108ED00001F0496FF7EC01F04A6F600EF5EC01F01C
:108EE0004B6FF7EC01F04C6FF7EC01F04D6FF7ECC6
:108EF00001F04E6F640EF5EC01F04F6FF7EC01F0EE
:108F0000506FF7EC01F0516FF7EC01F0526F680E03
:108F1000F5EC01F0536FF7EC01F0546FF7EC01F052
:108F2000556FF7EC01F0566F6C0EF5EC01F0010196
:108F3000686F6D0EF5EC01F0696F6E0EF5EC01F0E7
:108F40006B6F6F0EF5EC01F00501576FF7EC01F058
:108F5000586FF7EC01F0596FF7EC01F05A6F730E90
:108F6000F5EC01F05B6FF7EC01F05C6FF7EC01F0F2
:108F70005D6FF7EC01F05E6F770EF5EC01F05F6F5F
:108F8000F7EC01F0606FF7EC01F0616FF7EC01F0C6
:108F9000626F7B0EF5EC01F0636FF7EC01F0646F2C
:108FA000F7EC01F0656FF7EC01F0666F7F0EF5EC02
:108FB00001F0676FF7EC01F0686FF7EC01F0696F93
:108FC000F7EC01F06A6F830EF5EC01F06B6FF7ECD4
:108FD00001F06C6FF7EC01F06D6FF7EC01F06E6F64
:108FE000870EF5EC01F06F6FF7EC01F0706FF7ECA6
:108FF00001F0716FF7EC01F0726F8B0EF5EC01F080
:10900000736FF7EC01F0746FF7EC01F0756FF7EC2C
:1090100001F0766F8F0EF5EC01F001016C6F900E90
:10902000F5EC01F00501256F910EF5EC01F0EB6F09
:10903000F7EC01F0EC6F130EEE5D0001D8A02FEFFE
:1090400048F0D8A42BEF48F0890E0501ED5D000132
:10905000D8A02FEF48F00501EE6B320EED6F000146
:1090600001016B530001D8A438EF48F05BEC4AF0E3
:1090700001016B530001D8A449EF48F004EEA4F0BD
:109080001A0EF76E500EF66ED9EC02F0EF6A25EC70
:109090001EF0120004EEA4F01A0EF76E780EF66EB3
:1090A000D9EC02F0EF6A25EC1EF004EEA4F01A0EE3
:1090B000F76EB40EF66ED9EC02F0EF6A25EC1EF0F6
:1090C00004EEA4F01B0EF76E060EF66ED9EC02F05D
:1090D000EF6A25EC1EF004EEA4F01B0EF76E580E9E
:1090E000F66ED9EC02F0EF6A25EC1EF004EEA4F067
:1090F0001B0EF76EA00EF66ED9EC02F0EF6A25ECAF
:109100001EF004EEA4F01B0EF76EE80EF66ED9EC1E
:1091100002F0EF6A25EC1EF004EEA4F01C0EF76ED0
:10912000260EF66ED9EC02F0EF6A25EC1EF004EE86
:10913000A4F01C0EF76E640EF66ED9EC02F0EF6A26
:1091400025EC1EF004EEA4F01C0EF76E8C0EF66EED
:10915000D9EC02F0EF6A25EC1EF004EEA4F01C0E30
:10916000F76EB60EF66ED9EC02F0EF6A25EC1EF043
:1091700004EEA4F01C0EF76EF40EF66ED9EC02F0BD
:10918000EF6A25EC1EF004EEA4F01D0EF76E240E1F
:10919000F66ED9EC02F0EF6A25EC1EF004EEA4F0B6
:1091A0001D0EF76E580EF66ED9EC02F0EF6A25EC44
:1091B0001EF004EEA4F01D0EF76E8E0EF66ED9ECC6
:1091C00002F0EF6A25EC1EF004EEA4F01D0EF76E1F
:1091D000C20EF66ED9EC02F0EF6A25EC1EF004EE3A
:1091E000A4F01E0EF76E0A0EF66ED9EC02F0EF6ACE
:1091F00025EC1EF004EEA4F01E0EF76E2E0EF66E99
:10920000D9EC02F0EF6A25EC1EF004EEA4F01E0E7D
:10921000F76E560EF66ED9EC02F0EF6A25EC1EF0F2
:1092200004EEA4F01E0EF76E7E0EF66ED9EC02F080
:10923000EF6A25EC1EF004EEA4F01E0EF76ED00EC1
:10924000F66ED9EC02F0EF6A25EC1EF004EEA4F005
:109250001F0EF76E0E0EF66ED9EC02F0EF6A25ECDB
:109260001EF004EEA4F01F0EF76E6E0EF66ED9EC33
:1092700002F0EF6A25EC1EF004EEA4F01F0EF76E6C
:10928000B60EF66ED9EC02F0EF6A25EC1EF004EE95
:10929000A4F0200EF76E000EF66ED9EC02F0EF6A25
:1092A00025EC1EF004EEA4F0200EF76E300EF66EE4
:1092B000D9EC02F0EF6A25EC1EF004EEA4F0200ECB
:1092C000F76E6E0EF66ED9EC02F0EF6A25EC1EF02A
:1092D00004EEA4F0200EF76ECE0EF66ED9EC02F07E
:1092E000EF6A25EC1EF004EEA4F0210EF76E060ED8
:1092F000F66ED9EC02F0EF6A25EC1EF004EEA4F055
:10930000210EF76E760EF66ED9EC02F0EF6A25ECC0
:109310001EF004EEA4F0210EF76EC00EF66ED9EC2E
:1093200002F0EF6A25EC1EF004EEA4F0210EF76EB9
:10933000FE0EF66ED9EC02F0EF6A25EC1EF004EE9C
:10934000A4F0220EF76E500EF66ED9EC02F0EF6A22
:1093500025EC1EF004EEA4F0220EF76EA60EF66EBB
:10936000D9EC02F0EF6A25EC1EF004EEA4F0220E18
:10937000F76EEA0EF66ED9EC02F0EF6A25EC1EF0FD
:1093800004EEA4F0230EF76E300EF66ED9EC02F068
:10939000EF6A25EC1EF004EEA4F0230EF76E6E0EBD
:1093A000F66ED9EC02F0EF6A25EC1EF004EEA4F0A4
:1093B000230EF76EBA0EF66ED9EC02F0EF6A25ECCA
:1093C0001EF004EEA4F0230EF76EF80EF66ED9EC44
:1093D00002F0EF6A25EC1EF004EEA4F0240EF76E06
:1093E000400EF66ED9EC02F0EF6A25EC1EF004EEAA
:1093F000A4F0240EF76E820EF66ED9EC02F0EF6A3E
:1094000025EC1EF004EEA4F0240EF76EB60EF66EF8
:10941000D9EC02F0EF6A25EC1EF004EEA4F0240E65
:10942000F76EEE0EF66ED9EC02F0EF6A25EC1EF048
:1094300004EEA4F0250EF76E2C0EF66ED9EC02F0B9
:10944000EF6A25EC1EF004EEA4F0250EF76E5E0E1A
:10945000F66ED9EC02F0EF6A25EC1EF004EEA4F0F3
:10946000250EF76E900EF66ED9EC02F0EF6A25EC41
:109470001EF004EEA4F0250EF76ECE0EF66ED9ECBB
:1094800002F0EF6A25EC1EF004EEA4F0250EF76E54
:10949000FA0EF66ED9EC02F0EF6A25EC1EF004EE3F
:1094A000A4F0260EF76E280EF66ED9EC02F0EF6AE5
:1094B00025EC1EF0120004EEA4F0260EF76E6C0EE2
:1094C000F66ED9EC02F0EF6A25EC1EF001EE6DF0BD
:1094D000020E016E0501D751CCEC00F0EF6A04EEEC
:1094E000A4F0260EF76E940EF66ED9EC02F011EE93
:1094F0006DF0320EE75204E0E6CFEEFFE82EFAD729
:10950000EF6A000125EC1EF001EE6DF015EEDCF0C7
:10951000060EE75204E0E6CFEEFFE82EFAD7EF6A38
:1095200004EEA4F0260EF76EA40EF66ED9EC02F04F
:1095300011EE6DF0320EE75204E0E6CFEEFFE82EBA
:10954000FAD7EF6A25EC1EF001EE6DF0020E016E07
:10955000086AD9C521F0D8C520F0CFEC00F0EF6A39
:1095600004EEA4F0260EF76EB40EF66ED9EC02F0FF
:1095700011EE6DF0320EE75204E0E6CFEEFFE82E7A
:10958000FAD7EF6A25EC1EF001EE6DF0020E016EC7
:10959000086ADBC521F0DAC520F0CFEC00F0EF6AF5
:1095A00004EEA4F0260EF76EC40EF66ED9EC02F0AF
:1095B00011EE6DF0320EE75204E0E6CFEEFFE82E3A
:1095C000FAD7EF6A25EC1EF001EE6DF0020E016E87
:1095D0000501E551CCEC00F0EF6A04EEA4F0260E94
:1095E000F76ED40EF66ED9EC02F011EE6DF0320E7D
:1095F000E75204E0E6CFEEFFE82EFAD7EF6A00016B
:1096000025EC1EF001EE6DF0020E016E086AEEC54B
:1096100021F0EDC520F0CFEC00F0EF6A04EEA4F0ED
:10962000260EF76EE40EF66ED9EC02F011EE6DF038
:10963000320EE75204E0E6CFEEFFE82EFAD7EF6AEB
:1096400025EC1EF001EE6DF0020E016E086AF0C509
:1096500021F0EFC520F0CFEC00F0EF6A04EEA4F0AB
:10966000260EF76EF40EF66ED9EC02F011EE6DF0E8
:10967000320EE75204E0E6CFEEFFE82EFAD7EF6AAB
:1096800025EC1EF001EE6DF0020E016E086AF2C5C7
:1096900021F0F1C520F0CFEC00F0EF6A04EEA4F069
:1096A000270EF76E040EF66ED9EC02F011EE6DF097
:1096B000320EE75204E0E6CFEEFFE82EFAD7EF6A6B
:1096C00025EC1EF001EE6DF0020E016E086AF4C585
:1096D00021F0F3C520F0CFEC00F0EF6A04EEA4F027
:1096E000270EF76E140EF66ED9EC02F011EE6DF047
:1096F000320EE75204E0E6CFEEFFE82EFAD7EF6A2B
:1097000025EC1EF001EE6DF0020E016E086AF6C542
:1097100021F0F5C520F0CFEC00F0EF6A04EEA4F0E4
:10972000270EF76E240EF66ED9EC02F011EE6DF0F6
:10973000320EE75204E0E6CFEEFFE82EFAD7EF6AEA
:1097400025EC1EF001EE6DF0020E016E086AFCC5FC
:1097500021F0FBC520F0CFEC00F0EF6A04EEA4F09E
:10976000270EF76E340EF66ED9EC02F011EE6DF0A6
:10977000320EE75204E0E6CFEEFFE82EFAD7EF6AAA
:1097800025EC1EF001EE6DF0020E016E086AFEC5BA
:1097900021F0FDC520F0CFEC00F0EF6A04EEA4F05C
:1097A000270EF76E440EF66ED9EC02F011EE6DF056
:1097B000320EE75204E0E6CFEEFFE82EFAD7EF6A6A
:1097C00025EC1EF001EE6DF0020E016E086A00C677
:1097D00021F0FFC520F0CFEC00F0EF6A04EEA4F01A
:1097E000270EF76E540EF66ED9EC02F011EE6DF006
:1097F000320EE75204E0E6CFEEFFE82EFAD7EF6A2A
:1098000025EC1EF001EE6DF0020E016E086A02C634
:1098100021F001C620F0CFEC00F0EF6A04EEA4F0D6
:10982000270EF76E640EF66ED9EC02F011EE6DF0B5
:10983000320EE75204E0E6CFEEFFE82EFAD7EF6AE9
:1098400025EC1EF001EE6DF0020E016E086A04C6F2
:1098500021F003C620F0CFEC00F0EF6A04EEA4F094
:10986000270EF76E740EF66ED9EC02F011EE6DF065
:10987000320EE75204E0E6CFEEFFE82EFAD7EF6AA9
:1098800025EC1EF0D8960501E6A9D8860001D8B6C9
:1098900055EF4CF001EEA0F0270EF76E840EF66E39
:1098A000D9EC02F0EF6A5EEF4CF001EEA0F0270E6B
:1098B000F76E8E0EF66ED9EC02F0EF6A04EEA4F0AD
:1098C000270EF76E9A0EF66ED9EC02F011EEA0F0AC
:1098D000140EE75204E0E6CFEEFFE82EFAD7EF6A67
:1098E00025EC1EF0D8960501E6ABD8860001D8B667
:1098F00085EF4CF001EEA0F0270EF76EA80EF66E85
:10990000D9EC02F0EF6A8EEF4CF001EEA0F0270EDA
:10991000F76EB20EF66ED9EC02F0EF6A04EEA4F028
:10992000270EF76EBE0EF66ED9EC02F011EEA0F027
:10993000140EE75204E0E6CFEEFFE82EFAD7EF6A06
:1099400025EC1EF0D8960501E6ADD8860001D8B604
:10995000B5EF4CF001EEA0F0270EF76ECC0EF66ED0
:10996000D9EC02F0EF6ABEEF4CF001EEA0F0270E4A
:10997000F76ED60EF66ED9EC02F0EF6A04EEA4F0A4
:10998000270EF76EE20EF66ED9EC02F011EEA0F0A3
:10999000140EE75204E0E6CFEEFFE82EFAD7EF6AA6
:1099A00025EC1EF0D8960501E6AFD8860001D8B6A2
:1099B000E5EF4CF001EEA0F0270EF76EF00EF66E1C
:1099C000D9EC02F0EF6AEEEF4CF001EEA0F0270EBA
:1099D000F76EFA0EF66ED9EC02F0EF6A04EEA4F020
:1099E000280EF76E060EF66ED9EC02F011EEA0F01E
:1099F000140EE75204E0E6CFEEFFE82EFAD7EF6A46
:109A000025EC1EF0D896060109A1D8860001D8B62B
:109A100015EF4DF001EEA0F0280EF76E140EF66E65
:109A2000D9EC02F0EF6A1EEF4DF001EEA0F0280E27
:109A3000F76E1E0EF66ED9EC02F0EF6A04EEA4F09B
:109A4000280EF76E2A0EF66ED9EC02F011EEA0F099
:109A5000140EE75204E0E6CFEEFFE82EFAD7EF6AE5
:109A600025EC1EF0D896060109A9D8860001D8B6C3
:109A700047EF4DF004EEA4F0280EF76E380EF66EA8
:109A8000D9EC02F0EF6A25EC1EF052EF4DF004EE37
:109A9000A4F0280EF76E4E0EF66ED9EC02F0EF6AC7
:109AA00025EC1EF0D896060109ABD8860001D8B681
:109AB00067EF4DF004EEA4F0280EF76E660EF66E1A
:109AC000D9EC02F0EF6A25EC1EF072EF4DF004EED7
:109AD000A4F0280EF76E7C0EF66ED9EC02F0EF6A59
:109AE00025EC1EF004EEA4F0280EF76E940EF66E30
:109AF000D9EC02F0020E016E05019051CCEC00F0A1
:109B0000EF6A000125EC1EF0050177530001D8A48F
:109B100093EF4DF004EEA4F0280EF76EA40EF66E4F
:109B2000D9EC02F0EF6A010E0501775D0001D8A4BF
:109B3000A3EF4DF004EEA4F0280EF76EBC0EF66E07
:109B4000D9EC02F0EF6A020E0501775D0001D8A49E
:109B5000C0EF4DF004EEA4F0280EF76EE00EF66EA6
:109B6000D9EC02F0020E016E7BC52FF07AC52EF003
:109B700079C52DF078C52CF0030EFEEC00F0EF6AED
:109B800001016C530001D8A4D1EF4DF004EEA4F014
:109B9000280EF76EFA0EF66ED9EC02F0EF6A25EC9D
:109BA0001EF0010E01016C5D0001D8A4E3EF4DF041
:109BB00004EEA4F0290EF76E0E0EF66ED9EC02F04C
:109BC000EF6A25EC1EF001EE6DF0020E016E5AC533
:109BD0002FF059C52EF058C52DF057C52CF0030EA7
:109BE000FEEC00F0EF6A04EEA4F0290EF76E200EF2
:109BF000F66ED9EC02F011EE6DF0320EE75204E091
:109C0000E6CFEEFFE82EFAD7EF6A25EC1EF001EE64
:109C10006DF0020E016E6AC52FF069C52EF068C5A1
:109C20002DF067C52CF0030EFEEC00F0EF6A04EE99
:109C3000A4F0290EF76E300EF66ED9EC02F011EE9C
:109C40006DF0320EE75204E0E6CFEEFFE82EFAD7D1
:109C5000EF6A25EC1EF001EE6DF0020E016E4AC5B2
:109C60002FF049C52EF048C52DF047C52CF0030E46
:109C7000FEEC00F0EF6A04EEA4F0290EF76E400E41
:109C8000F66ED9EC02F011EE6DF0320EE75204E000
:109C9000E6CFEEFFE82EFAD7EF6A25EC1EF001EED4
:109CA0006DF0020E016E5EC52FF05DC52EF05CC535
:109CB0002DF05BC52CF0030EFEEC00F0EF6A04EE15
:109CC000A4F0290EF76E500EF66ED9EC02F011EEEC
:109CD0006DF0320EE75204E0E6CFEEFFE82EFAD741
:109CE000EF6A25EC1EF001EE6DF0020E016E6EC5FE
:109CF0002FF06DC52EF06CC52DF06BC52CF0030E4A
:109D0000FEEC00F0EF6A04EEA4F0290EF76E600E90
:109D1000F66ED9EC02F011EE6DF0320EE75204E06F
:109D2000E6CFEEFFE82EFAD7EF6A25EC1EF001EE43
:109D30006DF0020E016E4EC52FF04DC52EF04CC5D4
:109D40002DF04BC52CF0030EFEEC00F0EF6A04EE94
:109D5000A4F0290EF76E700EF66ED9EC02F011EE3B
:109D60006DF0320EE75204E0E6CFEEFFE82EFAD7B0
:109D7000EF6A25EC1EF001EE6DF0020E016E62C579
:109D80002FF061C52EF060C52DF05FC52CF0030EDD
:109D9000FEEC00F0EF6A04EEA4F0290EF76E800EE0
:109DA000F66ED9EC02F011EE6DF0320EE75204E0DF
:109DB000E6CFEEFFE82EFAD7EF6A25EC1EF001EEB3
:109DC0006DF0020E016E72C52FF071C52EF070C5D8
:109DD0002DF06FC52CF0030EFEEC00F0EF6A04EEE0
:109DE000A4F0290EF76E900EF66ED9EC02F011EE8B
:109DF0006DF0320EE75204E0E6CFEEFFE82EFAD720
:109E0000EF6A25EC1EF001EE6DF0020E016E52C5F8
:109E10002FF051C52EF050C52DF04FC52CF0030E7C
:109E2000FEEC00F0EF6A04EEA4F0290EF76EA00E2F
:109E3000F66ED9EC02F011EE6DF0320EE75204E04E
:109E4000E6CFEEFFE82EFAD7EF6A25EC1EF001EE22
:109E50006DF0020E016E66C52FF065C52EF064C56B
:109E60002DF063C52CF0030EFEEC00F0EF6A04EE5B
:109E7000A4F0290EF76EB00EF66ED9EC02F011EEDA
:109E80006DF0320EE75204E0E6CFEEFFE82EFAD78F
:109E9000EF6A25EC1EF001EE6DF0020E016E76C544
:109EA0002FF075C52EF074C52DF073C52CF0030E80
:109EB000FEEC00F0EF6A04EEA4F0290EF76EC00E7F
:109EC000F66ED9EC02F011EE6DF0320EE75204E0BE
:109ED000E6CFEEFFE82EFAD7EF6A25EC1EF001EE92
:109EE0006DF0020E016E56C52FF055C52EF054C50B
:109EF0002DF053C52CF0030EFEEC00F0EF6A04EEDB
:109F0000A4F0290EF76ED00EF66ED9EC02F011EE29
:109F10006DF0320EE75204E0E6CFEEFFE82EFAD7FE
:109F2000EF6A25EC1EF0050125530001D8A4A4EF2B
:109F30004FF004EEA4F0290EF76EE00EF66ED9ECA9
:109F400002F0EF6A25EC1EF0010E0501255D00010F
:109F5000D8A4B6EF4FF004EEA4F0290EF76EF60E7B
:109F6000F66ED9EC02F0EF6A25EC1EF012004AEC16
:049F700048F01200A3
:020000040030CA
:03000100861A0F4D
:020005008181F7
:060008000FC00FE00F40E5
:00000001FF
